:106F56000000090200000301FA0400EF0500030A1D
:106F66000A5A0B001E0C00FA0D00030E00040F0156
:106F760064100096120132130AFA14010217010A6C
:106F86001801EF1905321A010A1B01EF1C05321F01
:106F9600FFFF20FFFF23011E2400642A00FA2B00B6
:106FA600FA2C50782D003D2E004630006432507881
:106FB6003300003432FF350164360164370150383E
:106FC6000A643A00033B00043C00643E003C3F0078
:106FD6000140FFFF411450420A5A430AC844053291
:106FE6004500B44600FA4900024B00014C00FA5035
:106FF6000808510596520A32530B46540A9657050D
:1070060046590A465A32FA5B010A5C0A325E000A9F
:107016005F00646200FE64011167FFFF6801016999
:1070260001016A05966B00006C32FF6D0004730067
:10703600007400007801327901327EFFFF7FFFFF86
:1070460080FFFF81FFFF8400648800028A00019DA3
:107056000A969E00019FFFFFA00124A2000AA3FF3B
:10706600FFA40064A50064A6FFFFA7FFFFA8FFFF1B
:10707600A9FFFF0101241500022F003C47014848E3
:1070860002045600004EFFFF58000261FFFF660033
:10709600028500AF8600018700FA89010A99000877
:1070A600A100FAFAFAFA0101241500022F1E3C4744
:1070B60001484802045600004EFFFF58000261FFD7
:1070C600FF6600028500AF8600018700FA89010A83
:1070D600990000A10000FAFAFA0065006F00790035
:1070E60083008D009700A100AC00B600C000CA0066
:1070F600D400DE00E800F20058006000680070006E
:1071060078008000880090009800A000A800B000D9
:10711600B800C100C800D000D800DF00E600EE00CD
:10712600F600410047004D00530059005F0065001E
:107136006C00710077007D00830089008F00950048
:107146009B00A200A700AC00B200B900C000C500B9
:0D715600CA00D200D500DD00E100E700EF27
:103D750085F97485FA757E017F00E575127275E522
:103D8500742FFF50010E8E5A8F5B90001CE0FCA330
:103D9500E0FDEF2DFDEE3CFC8C5C8D5D90003CE084
:103DA500FAA3E0FBED2BFBEC3AFA8A5C8B5D2275FE
:103DB500A71085F97485FA757E017F00E575127285
:103DC50075E5742FFF50010E8E5A8F5B9000F6E05B
:103DD500B40210AC2DAD2EEF2DFDEE3CFC8C5C8DB0
:103DE5005D8016AE5AAF5B90001CE0FCA3E0FDEFD2
:103DF5002DFDEE3CFC8C5C8D5DAE5CAF5D90003CBA
:103E0500E0FCA3E0FDEF2DFDEE3CFC8C5C8D5D221E
:103E1500E55DF5FBE55CF5FCD29322E55DF5E9E5AD
:103E25005CF5EAD29422E55DF5EBE55CF5ECD29123
:103E350022E55DF5EDE55CF5EED292229000D8E045
:103E4500C394045003123DB4E55DF5FBE55CF5FC58
:103E5500D287229000D8E0C394045003123DB4E504
:103E65005DF5E9E55CF5EAD290229000D8E0C394CF
:103E7500045003123DB4E55DF5EBE55CF5ECE5B505
:103E85004410F5B5229000D8E0C394045003123DC8
:103E9500B4E55DF5EDE55CF5EEE5B54420F5B52257
:103EA500A203B34004D2A08002C2A022E50C906B0D
:103EB5003FF8282873023F5E75E700A239B3400832
:103EC500E5B54408F5B58006E5B554F7F5B575E7EC
:103ED50010023F5E023F5EA23992A0807CA2399219
:103EE500978076A23992A28070A23992A1806A75D4
:103EF500E700A239B34008E5B54440F5B58006E5CD
:103F0500B554BFF5B575E710804F75E700A239B315
:103F15004008E5B54480F5B58006E5B5547FF5B5AF
:103F250075E710803475E700A239B34008E5B5445C
:103F350010F5B58006E5B554EFF5B575E7108019B0
:103F450075E700A239B34008E5B54420F5B580060C
:093F5500E5B554DFF5B575E71080
:106B3F00023EBA023EBD023ED9023EDC023EE202F6
:106B4F003EE8023EEE023EF4023F0F023F2A023FB2
:016B5F0045F0
:103F5E00227433900167F07436900168F0742D90DE
:103F6E000169F0743190016AF0742090016BF07465
:103F7E005690016CF0743890016DF0742090016EC3
:103F8E00F0743290016FF07443900170F0746F9082
:103F9E000171F07469900172F0746C900173F07499
:103FAE0020900174F07420900175F02290089EE02C
:103FBE00FEA3E0FF7423D39F74019E400C906F56B6
:103FCE00120048E493F599802E90F802E493B4051C
:103FDE001490089EE0FEA3E0FF906F89120048E463
:103FEE0093F599801290089EE0FEA3E0FF906F5625
:103FFE00120048E493F59990089E12728390089EE1
:10400E00E0FEA3E0FFEFB45607EEB40103754E00D9
:10401E0022AE5AAF5B740A8E048F05FF1272658C46
:10402E005C8D5DAE5AAF5B740A8E048F05FF127203
:10403E00908C5A8D5BE55B455A6013740AC3955B91
:10404E00FFE4955AFE8E5A8F5B785C1272C8E57447
:10405E00A85CB80015D3955D4010E574C3955DFF5F
:10406E00E4955CFE8E5C8F5D8010E5742424C39510
:10407E005DFFE4955CFE8E5C8F5DAE5CAF5D74247F
:10408E006F4E700B755D23755C0075740180037542
:10409E007400229000A4E0B40104C2078002D2078B
:1040AE009000A5E0B40104C2088002D2089000E29C
:1040BE00E075F0E1A4FFAEF0740A8E048F05FF12D6
:1040CE007265900892ECF0A3EDF09000E2E075F0CE
:1040DE002BA4FFAEF0900018EEF0A3EFF07E017F60
:1040EE00009000A0E01272759000E3E08E048F0540
:1040FE00FF127265740AFF1272658D619000ECE01A
:10410E0075F0E1A4FFAEF0740A8E048F05FF1272F3
:10411E0065900896ECF0A3EDF09000EEE060139041
:10412E0000EEE0F5F0741684FF7E00EF9008F4F0D8
:10413E00800674649008F4F09000E4E0900081F042
:10414E00900130E090008BF0900132E0FE9000E0A4
:10415E00E08E0088F0A4FFAEF0EF9008FDF0900125
:10416E000BE075F013A4FDACF090003CECF0A3ED69
:10417E00F0A225B3401690017CE0700C90017DE01A
:10418E00700690017EE060028002C22590017CE004
:10419E00B4300F90017DE0B4470890017EE0643B9F
:1041AE0060028004D2268002C22690009DE0FE901E
:1041BE0008FEE06E601A7599E612019C74AB9000D1
:1041CE005BF01206DA75096475080012062480FE8B
:1041DE00900095E0700674009000CAF0900085E0A3
:1041EE00FE9000CAE0B5063F900087E0FE9000E822
:1041FE00E0B50633900086E0FE9000F6E0B50627A7
:10420E00900089E0FE90009DE0B5061B900088E0CE
:10421E00FE9000D8E0B5060F90008AE0FE900116E1
:10422E00E06E70030243EC9000D8E0D39402500687
:10423E009000F6E060087408900119F08006740A88
:10424E00900119F09000D8E0D3940240089000F647
:10425E00E064026002800674009000F6F090009D0B
:10426E00E0B40106740090009DF090009DE0B40251
:10427E000674009000E8F090009DE0B40306740010
:10428E009000F5F0900116E06014742990078EF0FE
:10429E0074009006D6F074009006D7F0800C74006F
:1042AE0090078EF074299006D6F09000F6E0B401D7
:1042BE0014741790011CF074009006DEF0740090D8
:1042CE0006DFF0800C740090011CF074179006DE6F
:1042DE00F09000E8E0D394014014741890011BF0A4
:1042EE0074009006E2F074009006E3F0800C740007
:1042FE0090011BF074189006E2F09000CAE0B40230
:10430E001474199000B2F074009006E6F0740090E8
:10431E0006E7F0800C74009000B2F074199006E677
:10432E00F09000CAE06014741A9000B1F07400901E
:10433E0006EAF074009006EBF0800C74009000B169
:10434E00F0741A9006EAF09000D8E0B402069000DD
:10435E00F6E06002802674079006F6F07408900668
:10436E00FAF0740090078AF0740090078BF07400D6
:10437E0090078CF0740090078DF0803074009006DA
:10438E00F6F074009006F7F074009006FAF07400E0
:10439E009006FBF0740590078AF0740690078BF078
:1043AE00740790078CF0740890078DF0D22490005B
:1043BE00CAE0900085F09000F6E0900086F0900044
:1043CE00E8E0900087F09000D8E0900088F0900030
:1043DE009DE0900089F0900116E090008AF0900127
:1043EE0000E0B40117900028740FF0A374FFF09052
:1043FE00002AE4F0A3F07402900100F0900100E0B6
:10440E00B4034190002AE0FEA3E0FF900028E0FCF8
:10441E00A3E0FD1272C07410127275740812003986
:10442E00EF9000FFF0EF700674FF9000FFF0740045
:10443E00900100F0900029E09000B6F0900028E086
:10444E009000B7F0900091E090008EF0900090E018
:10445E0090008DF09000BFE0C3941E50569000BFA8
:10446E00E0F404241E90008FF090008FE075F00AA7
:10447E0084FF7E008F7490008FE075F00A84ADF09B
:10448E007C008D7590008DE0D39575400D90008D5C
:10449E00E0C3957590008DF0800F90008DE0240A9A
:1044AE00C3957590008DF0057490008EE025749084
:1044BE00008EF090008EE090004EF090004EE0D313
:1044CE009424400B90004EE0C3942490004EF09044
:1044DE00004EE0240990004FF090004EE024129020
:1044EE000050F090004EE0241B900051F090004FD1
:1044FE00E0D39424400B90004FE0C3942490004FDF
:10450E00F0900050E0D39424400B900050E0C39400
:10451E0024900050F0900051E0D39424400B900072
:10452E0051E0C39424900051F0900056E4F09000B6
:10453E004EE0B4240C9000567401F090004E7401BD
:10454E00F0900057E4F090004FE0B4240C90005728
:10455E007401F090004F7401F0900058E4F0900058
:10456E0050E0B4240C9000587401F0900050740187
:10457E00F0900059E4F0900051E0B4240C900059F2
:10458E007401F09000517401F0900091E0FE9000E3
:10459E00F4E02E90005CF090005CE06412600790F6
:1045AE00005CE0B4240690005CE004F090005CE057
:1045BE00D39424400B90005CE0C3942490005CF0F4
:1045CE0090005CE0D39412400D90005CE0C3941216
:1045DE0090005DF0800A90005CE0241290005DF087
:1045EE00755E12900091E0FE9000D7E0D39E5013BE
:1045FE00900091E0FE9000D7E0F4042E049000525B
:10460E00F08013900091E02424FE9000D7E0F40493
:10461E002E04900052F0900052E075F00984AFF035
:10462E007E00EF4E7006900052E004F0900052E0D3
:10463E00B425069000527401F0900052E0D39424F9
:10464E00400F900052E0C39424900052F0D21F808D
:10465E0002C21F900052E02409900053F0900052C5
:10466E00E02412900054F0900052E0241B9000556C
:10467E00F0900053E0D39424400B900053E0C39489
:10468E0024900053F0900054E0D39424400B9000FB
:10469E0054E0C39424900054F0900055E0D3942439
:1046AE00400B900055E0C39424900055F012019CED
:1046BE0022C293C294C291C292C287C290E5B554EF
:1046CE00EFF5B5E5B554DFF5B5C296C295C2A0C2F9
:1046DE0097C2A2C2A1E5B554BFF5B5E5B5547FF5B5
:1046EE00B5E5B554FBF5B5C209755F469000DAE045
:1046FE007005756E028003756E0375550075540056
:10470E0090001074FFF0A374DCF0C210C212C21439
:10471E00C21674C890003EF074C8900042F074C87F
:10472E00900046F074C890004AF075530075520020
:10473E00C204754700E570B413037570007564000C
:10474E0090001EE4F0A3F0757110C20CC20DC20EE3
:10475E00C20FC203755700755600900012E4F0A305
:10476E00F0900014E4F0A3F0C229755900755800BA
:10477E0090009CE075F032A4FFAEF0900026EEF0B3
:10478E00A3EFF090008CE4F09008FAE4F0C227D288
:10479E001CC21BD21DC21EC21FC220900016E4F006
:1047AE00A3F022755B00755A00AE5AAF5B7422C33C
:1047BE009F74019E50030248A5906F56120048E464
:1047CE0093645F6023906F56120048E493647E609A
:1047DE0017906F56120048E4936481600B906F56E9
:1047EE00120048E493B48403024885AE5AAF5B903E
:1047FE006F56120048E4939000901272A60FBF00FD
:10480E00010EE0FC906F56120048ECFEE493FFEEB2
:10481E00C39F5026AE5AAF5B0FBF00010E906F566E
:10482E00120048AE5AAF5BE493FC906F56120048EC
:10483E00E4939000901272A6ECF0AE5AAF5B906FBC
:10484E0056120048E4939000901272A6E0FC906F0E
:10485E0058120048ECFCE493FDECD39D4019906F88
:10486E0058120048E493FC906F56120048E493905F
:10487E0000901272A6ECF0AE5AAF5B74022FFF508E
:10488E00010E8E5A8F5B785B740126F6500418E485
:10489E0036F640030247B722755B00755A00AE5AD2
:1048AE00AF5B7432BE00039F500302497390707960
:1048BE00120048E4939000901272A60FBF00010EF2
:1048CE00E0FC907079120048ECFEE493FFEEC39F7B
:1048DE005026AE5AAF5B0FBF00010E9070791200DA
:1048EE0048AE5AAF5BE493FC907079120048E493A3
:1048FE009000901272A6ECF0AE5AAF5B90707912E7
:10490E000048E4939000901272A6E0FC90707B1227
:10491E000048ECFCE493FDECD39D401990707B12A3
:10492E000048E493FC907079120048E49390009054
:10493E001272A6ECF0AE5AAF5B742D6F4E70067508
:10494E005B33755A00AE5AAF5B74022FFF50010EE7
:10495E008E5A8F5B785B740126F6500418E436F697
:10496E0040030248AC22755B00755A00AE5AAF5B2D
:10497E007432BE00039F5003024A419070AC120085
:10498E0048E4939000901272A60FBF00010EE0FC57
:10499E009070AC120048ECFEE493FFEEC39F5026DD
:1049AE00AE5AAF5B0FBF00010E9070AC120048AE56
:1049BE005AAF5BE493FC9070AC120048E493900005
:1049CE00901272A6ECF0AE5AAF5B9070AC1200482B
:1049DE00E4939000901272A6E0FC9070AE12004824
:1049EE00ECFCE493FDECD39D40199070AE120048A0
:1049FE00E493FC9070AC120048E493900090127215
:104A0E00A6ECF0AE5AAF5B742D6F4E7006755B332D
:104A1E00755A00AE5AAF5B74022FFF50010E8E5ABC
:104A2E008F5B785B740126F6500418E436F640036B
:104A3E0002497A2285F97485FA757E017F00E57543
:104A4E00127275E5742FFF50010E8E5A8F5BAC5C9F
:104A5E00AD5DEF2DFDEE3CFC8C5C8D5D123E1512B6
:104A6E003E20123E2B123E369000D8E0D3940240E8
:104A7E002C75A71085F97485FA757E017F00E57592
:104A8E00127275E5742FFF50010E8E5A8F5B123E17
:104A9E0041123E58123E6F123E8A75A7002275A72C
:104AAE001085F97485FA757E017F00E575127275B1
:104ABE00E5742FFF50010E8E5A8F5B7E017F76902C
:104ACE000115E0127275AC5AAD5BED2FFFEC3EFE98
:104ADE008E5C8F5DE55DF5FDE55CF5FE900081E495
:104AEE00F075A700741290005FF02285F97485FAB4
:104AFE00757E017F00E575127275E5742FFF50010A
:104B0E000E8E5A8F5B900018E0FCA3E0FDEF2DFD9A
:104B1E00EE3CFC8C5C8D5DE55DF5FDE55CF5FE2205
:104B2E00056522A2D8B34002C293A2D9B34002C2F5
:104B3E0094A2DAB34002C291A2DBB34002C292A2A7
:104B4E00DCB34018A2965006741990005FF0A2953F
:104B5E005006741990005FF0C296C29575D8402227
:104B6E0085A77375A710A2D8B34002C287A2D9B386
:104B7E004002C290A2DAB34006E5B554EFF5B5A2F5
:104B8E00DBB34006E5B554DFF5B5A2DCB3400890C3
:104B9E0000E4E0900081F075D8408573A72290F86C
:104BAE0000E4936406600280FE12009E75A70075F5
:104BBE00D80075D90475DA0975DB0975DC0975DD60
:104BCE000975DE0975D84075A71075D80075D9041A
:104BDE0075DA0975DB0975DC0975DD0975DE097590
:104BEE00D84075A7001200FB7509C875080012069B
:104BFE002475A70FE5FC90006EF0E5FB90006FF0BA
:104C0E00E5FA900070F0E5F9900071F075A700904C
:104C1E00F800E493F5281207439008A7E0D3940315
:104C2E0050079008A7E0B4010674009008A7F09012
:104C3E0008A7E09008FEF074019000D9F09008A744
:104C4E00E0906B60F8282873802A802875A70F756E
:104C5E00F30F75A700A2A3400674029000D9F0804E
:104C6E001375A70F75F31775A700A2A4400674025B
:044C7E009000D9F0D9
:0C6B6000024C56024C58024C5A024C6F7A
:104C82009000D9E0B4022AC21A120AEC740290000F
:104C9200D9F09008A7E0906B6CF8282873801080F8
:0F4CA2000E74009000E8F0800674009000F5F0AA
:0C6B6C00024C9F024CA1024CA3024CAB57
:104CB1008028D21A120A0174019000D9F09008A735
:104CC100E0906B78F82828738010800E74009000B3
:0A4CD100E8F0800674009000F5F092
:0C6B7800024CC9024CCB024CCD024CD5A3
:104CDB0090F807E49390007BF090007BE044089001
:104CEB00007BF090007BE054FE90007BF01203BD44
:104CFB00123F5F9008B4E090017CF09008B5E09013
:104D0B00017DF09008B6E090017EF090017CE070A0
:104D1B000C90017DE0700690017EE060028004C281
:104D2B00258002D2259000CAE004900085F0900106
:104D3B0034E0B4FF067400900134F0900135E0B418
:104D4B00FF067400900135F01247B190F802E4931E
:104D5B00B4050512497480031248A6740090010033
:104D6B00F01240A1E5B54401F5B57406900061F071
:104D7B007400900062F07401900063F090F802E40C
:104D8B0093900064F090F803E493900065F090F832
:104D9B0004E493900066F07406900067F090006452
:104DAB00E0B405067405900067F0743C900068F061
:104DBB007403900069F0740790006AF0740190001E
:104DCB006BF090F805E49390006CF090F806E49388
:104DDB0090006DF07400900075F07400900076F008
:104DEB007400900077F07400900078F074009000DD
:104DFB0079F0740090007AF074FF90007CF0A2B60A
:104E0B00B39205A2B3B39206A2A4B39222A2A3B308
:104E1B00922390007DE4F0757000743A900790F047
:104E2B0074FD900791F090007EE4F0756F01900097
:104E3B005FE4F09000DAE0B40106741A90005FF0C2
:104E4B00C221756400C20AD20BC203757200C22460
:104E5B001205C6756000756C00756200756632755B
:104E6B006700756800756900756A00756B009000C6
:104E7B001EE4F0A3F0756D00D2B2D2A4D2B0D2B1C1
:104E8B00D2A3D2A7D2A6D2A5D2B77E017F00900023
:104E9B00B7E01272759000B6E02FFF50010E900034
:104EAB0028EEF0A3EFF0EFD394FFEE940F400790B2
:104EBB000028E4F0A3F09000FFE0700674FF900070
:104ECB00FFF09000DAE07005756E028003756E03DB
:104EDB00740090011DF0740090011EF0742A900173
:104EEB001FF07400900120F074009006DAF0741B30
:104EFB009006EEF0741C9006F2F0741590077EF09D
:104F0B00741690077FF07400900780F07400900780
:104F1B0081F07400900782F07400900783F07400A6
:104F2B00900784F07400900785F07401900786F069
:104F3B007402900787F07403900788F0740490074D
:104F4B0089F0740590078AF0740690078BF0D29C59
:104F5B00E571D3941040037571109006D7E0D3948C
:104F6B000C400674009006D7F09006DFE0D3940C4B
:104F7B00400674009006DFF09006E3E0D3940C40FB
:104F8B000674009006E3F09006E7E0D3940C40061D
:104F9B0074009006E7F09006EBE0D3940C40067497
:104FAB00009006EBF09006EFE0D3940C40067400F3
:104FBB009006EFF09006F3E0D3940C40067400904B
:104FCB0006F3F09006F7E0D3940C400674009006BD
:104FDB00F7F09006FBE0D3940C400674009006FBB0
:104FEB00F0D2EC75CF01A298B34005C298120C54C5
:104FFB00E54E6006A299B3B340028005C299121028
:10500B00E0E54F64016005E54FB4040280D5C28E24
:10501B007E107F00E565127275E58D75F010A4FDAD
:10502B00ACF0EF2DFDEE3CFCE58B75F01084FF7EB4
:10503B0000ED2FFFEC3EFE8E548F55D28E9000BDAF
:10504B00E060099000BDE0C3943D4002805C90009D
:10505B0020127283900020E0FEA3E0FF900022E07C
:10506B00FCA3E0FDEFB50542EEB5043EB218A20479
:10507B00B3401975E700A218B34008E5B54404F531
:10508B00B58006E5B554FBF5B575E710900022E049
:10509B00FEA3E0FF900024E0FCA3E0FDEF2DFDEE6E
:1050AB003CFC900022ECF0A3EDF09000CAE060090C
:1050BB009000CAE0C3940340028061123027A2041F
:1050CB0040089000B4E0F546801BE560C395615045
:1050DB0005754600800F9000A1E0C39562500690C5
:1050EB0000C7E0F546E54675F002A4FFAEF0900868
:1050FB009CEEF0A3EFF0AC2FAD30EDD39FEC9E40C8
:10510B0004C2A1800B90007DE0C394415002D2A158
:10511B009000CAE0B40205A2A1B392A29000CAE02B
:10512B00B4031C123142AE2FAF3090089CE0FCA3AD
:10513B00E0FDEFD39DEE9C4004D2A18002C2A19072
:10514B0000A5E06009A2B3300601B3B3400280565C
:10515B00A2B3300601B3404EA2B3300801B34039BD
:10516B00A21C403090008BE0D3955F40259008FA4D
:10517B00E0701390008CE0B401069008FA7401F013
:10518B0090008CE004F0A21BB3400590008CE4F07F
:10519B00D21BD21CA208B39206A208B330B301B340
:1051AB004004A2089206A2B6300501B35003025880
:1051BB004EA2B6300501B3500302584EA2B63007CB
:1051CB0001B3500302571E756F009000BDE0B43D54
:1051DB001975E700A207B34008E5B554FBF5B58098
:1051EB0006E5B54404F5B575E710055FA209B3B341
:1051FB005013AE54AF55900010E0FCA3E0FDEDC38F
:10520B009FEC9E40030253CBE56EB4032EA229B351
:10521B004022E55FB42403756E01E55FC39424500F
:10522B000690005F7401F0E55FD39424400674028E
:10523B0090005FF0755F01D229805EE56EB4020AC3
:10524B00756E01755F24C21BC21DE55FB424057525
:10525B005F01804590005FE07030E55FC3942450A0
:10526B000690005F7401F0E55FD39424400674024E
:10527B0090005FF0E55FC394245002D221E55FD329
:10528B0094244002D221C296C2959000DAE0B40178
:10529B00051246BF8003755F01AE56AF57AC54ADD8
:1052AB0055EF2DFDEE3CFC7403FF1272658C568D91
:1052BB00579000BDE060099000BDE0C3943D4002F3
:1052CB008049900020E0FEA3E0FF9000BDE08E043B
:1052DB008F05FF12726574018C068D0712003990D1
:1052EB000024EEF0A3EFF0900024E0F8A3E0900090
:1052FB0022C8F0A3C8F0900020E4F0A3F0C2187508
:10530B00E700E5B554FBF5B575E710A2A4B3400271
:10531B00C222A2A3B34002C223A221B34002C221E4
:10532B00B21E9008FAE0B40111A21BB34004D21EC6
:10533B008002C21E74029008FAF09008FAE0C3943F
:10534B00025006A204B3B34002800674029008FA1E
:10535B00F09000D8E0B404629000A5E060069008DD
:10536B00FAE07002800DA21D301B01B340059000C6
:10537B008CE4F09000DAE064016006A227B3B3502E
:10538B00179000A5E06009A21B301D01B3B34002CA
:10539B008006740590005FF0B21DA21CB3401BA2E7
:1053AB001BB34004D21D8002C21D9000DAE07006D0
:1053BB009008FAE070028002D227C21BC21C803A0E
:1053CB00AE56AF57AC54AD55EF2DFDEE3CFC740112
:1053DB008C068D071200398E568F57E56EC39402DB
:1053EB00500DAC54AD557488C39D74139C40028012
:1053FB00091246BF740690005FF0E55FB424127487
:10540B000390005FF0D2219000DAE0B40103124662
:10541B00BFAE58AF59AC54AD55EF2DFDEE3CFC8CE7
:10542B00588D59AE54AF55EFD39DEE9C4011900063
:10543B0016E0FAA3E0FBEBC394E8EA940340028086
:10544B0006900016127283900014E0FEA3E0FFACEE
:10545B0054AD55EF2DFDEE3CFC900014ECF0A3ED9C
:10546B00F09000DAE0B4011DAE54AF557405127222
:10547B007574038E048F05FF127265900010ECF0AB
:10548B00A3EDF08016AE54AF557403127275740110
:10549B00120039900010EEF0A3EFF0C28E758D0064
:1054AB00758B00756500755501755400D28EE55FDF
:1054BB00240875F00984AFF07E00EF4E60030255AF
:1054CB004EE56E6013AE56AF5774091272759000AD
:1054DB0012EEF0A3EFF0800F900014E0F8A3E09031
:1054EB000012C8F0A3C8F0900012E0FEA3E0FFEF9B
:1054FB004E600B7C7E7DB61271638E528F53900083
:10550B0014E4F0A3F0AE52AF537428BE00039F50C7
:10551B0010E5642FFF50010E74011200398E528F6B
:10552B00538553649000E1E0A852B8000DD3955316
:10553B004008E55390005EF080099000E1E0149084
:10554B00005EF09000D8E0B40408900052E0655F74
:10555B006002800EA21E301F01B34004D2208002D5
:10556B00C220E55F640B6005E55FB41D099000CABE
:10557B00E06003122CDD90005CE0655F600790003B
:10558B005DE0B55F03757000A20AB35006A209B3C4
:10559B00B34003025646900096E0B4017390011895
:1055AB00E0B40214121281900082E075F0BCA4FFEB
:1055BB00AEF08E5C8F5D8056E56875F00A84FF7ED9
:1055CB0000900590120048E0F55B755A00AE5AAF9B
:1055DB005B9000BBE012727574648E048F05FF1232
:1055EB0072658C5C8D5DE55D90005AF0AE5AAF5BD9
:1055FB00900094E012727574648E048F05FF127222
:10560B006574BC8C068D071272758E5C8F5D80176E
:10561B00900094E075F0BCA4FFAEF08E5C8F5D90B3
:10562B0000BBE090005AF0E562C394CC5006E55DF8
:10563B00455C70028003124A42D20AE56EB4010641
:10564B00E55F640B6002800C757100900060740163
:10565B00F0756E00E56E60030257199000DDE06097
:10566B000D900081E0A852B8000695534002804887
:10567B009000DDE0B4022790004EE0655F6017906C
:10568B00004FE0655F600F900050E0655F60079032
:10569B000051E0B55F03757103756D00800CC2019D
:1056AB00756D0090001EE4F0A3F0900081E06006A1
:1056BB00740990005FF0805690004EE0655F6017B4
:1056CB0090004FE0655F600F900050E0655F6007F2
:1056DB00900051E0B55F3775710090004EE0B55FFB
:1056EB00069000607401F090004FE0B55F06740205
:1056FB00900060F0900050E0B55F0674039000607E
:10570B00F0900051E0B55F067404900060F0A207C2
:10571B00B39205A207B330B601B3500302584E75CE
:10572B006F019000BDE0B43D1975E700A207B340CF
:10573B0008E5B54404F5B58006E5B554FBF5B5753C
:10574B00E71075E700E5B54401F5B575E710742B67
:10575B0090007DF0A2079205E55FD3944A4014D2E6
:10576B0009E55FD3946E400B740590005FF0D22176
:10577B00755F4675E700900113E0A852B80005D39A
:10578B009553500D900112E0A852B8000495535058
:10579B00028008E5B54402F5B58017900114E0D3FB
:1057AB0095624008E5B54402F5B58006E5B554FDB4
:1057BB00F5B575E7109000E5E0B40107E56BC39410
:1057CB004140028018E56BC3941450087413900089
:1057DB005FF08006740E90005FF01246BF9000677A
:1057EB00E0FE900064E0C39E4009900064E0D39417
:1057FB0008400974FB90005FF01246BF900065E013
:10580B006015900065E0FE900063E06E600974FC2B
:10581B0090005FF01246BF900066E0601590006646
:10582B00E0FE900068E06E600974FE90005FF0127D
:10583B0046BF9008A7E06006900115E06002800368
:10584B00120BD7A221B34004C296C295900115E06A
:10585B00600CAE52AF537414BE00059F40028037EC
:10586B0090009DE0906B84F8282873802A8028A2F2
:10587B00A3B35005A223B340028005124AACD22336
:10588B008015A2A4B35005A222B340028005124A90
:07589B00ACD2228002800064
:106B840002587602587802587A02588D0258A002A8
:026B940058A205
:1058A200A20CB3B35008900052E0655F6003025A45
:1058B20028A202B35006A201B3B34003025A2090B9
:1058C20000D8E0B4040280030259DD9008FAE0B483
:1058D200020280030259C2A220B3406A123D7590AF
:1058E2000129E0601F90001CE0FEA3E0FF9001216F
:1058F200E012727574C88E048F05FF1272658C5C9B
:105902008D5D800A90001CE0F55CA3E0F55DAE5C65
:10591200AF5D745E12727574058E048F05FF12728C
:1059220065AE5AAF5BED2FFFEC3EFE8E5C8F5D9055
:10593200003CE0FCA3E0FDEF2DFDEE3CFC8C5C8D19
:105942005D123E15806E123DB4900129E0D394049D
:10595200401F90001CE0FEA3E0FF900125E01272C0
:105962007574C88E048F05FF1272658C5C8D5D8024
:105972000A90001CE0F55CA3E0F55DAE5CAF5D74DF
:105982005E12727574058E048F05FF127265AE5A2F
:10599200AF5BED2FFFEC3EFE8E5C8F5D90003CE036
:1059A200FCA3E0FDEF2DFDEE3CFC8C5C8D5D123E18
:1059B2004175A7009000F6E0B40103123EA58019DC
:1059C200123D75123E15123DB4123E4175A700906C
:1059D20000F6E0B40103123EA58043123D75123E6B
:1059E200159000D8E0B4031275A710123E41900042
:1059F200F6E0B40103123EA5802175A7109000F6CF
:105A0200E0B40106A203B3B340028005123E418016
:105A12000A9000F6E0B40203123E4175A700C20CE0
:105A2200D20DD20ED20FA20DB3B35008900053E0A4
:105A3200655F6003025BB1A202B35006A201B3B379
:105A42004003025BA99000D8E0B404028003025B29
:105A5200669008FAE0B402028003025B4BA220B314
:105A6200406D123D75900129E0D39401401F9000D2
:105A72001CE0FEA3E0FF900122E012727574C88E52
:105A8200048F05FF1272658C5C8D5D800A90001C8C
:105A9200E0F55CA3E0F55DAE5CAF5D745E1272751D
:105AA20074058E048F05FF127265AE5AAF5BED2F3F
:105AB200FFEC3EFE8E5C8F5D90003CE0FCA3E0FDBF
:105AC200EF2DFDEE3CFC8C5C8D5D123E20806E1253
:105AD2003DB4900129E0D39405401F90001CE0FEE4
:105AE200A3E0FF900126E012727574C88E048F0540
:105AF200FF1272658C5C8D5D800A90001CE0F55C83
:105B0200A3E0F55DAE5CAF5D745E12727574058ED6
:105B1200048F05FF127265AE5AAF5BED2FFFEC3EAC
:105B2200FE8E5C8F5D90003CE0FCA3E0FDEF2DFD5E
:105B3200EE3CFC8C5C8D5D123E5875A7009000F621
:105B4200E0B40103123EA58019123D75123E2012E7
:105B52003DB4123E5875A7009000F6E0B40103125E
:105B62003EA58043123D75123E209000D8E0B4035A
:105B72001275A710123E589000F6E0B40103123ECF
:105B8200A5802175A7109000F6E0B40106A203B328
:105B9200B340028005123E58800A9000F6E0B4023B
:105BA20003123E5875A700D20CC20DD20ED20FA21C
:105BB2000EB3B35008900054E0655F6003025D3A93
:105BC200A202B35006A201B3B34003025D329000B9
:105BD200D8E0B404028003025CEF9008FAE0B40259
:105BE200028003025CD4A220B3406D123D75900185
:105BF20029E0D39403401F90001CE0FEA3E0FF9035
:105C02000123E012727574C88E048F05FF1272654B
:105C12008C5C8D5D800A90001CE0F55CA3E0F55D74
:105C2200AE5CAF5D745E12727574058E048F05FFF3
:105C3200127265AE5AAF5BED2FFFEC3EFE8E5C8FAB
:105C42005D90003CE0FCA3E0FDEF2DFDEE3CFC8C02
:105C52005C8D5D123E2B806E123DB4900129E0D323
:105C62009406401F90001CE0FEA3E0FF900127E095
:105C720012727574C88E048F05FF1272658C5C8D6A
:105C82005D800A90001CE0F55CA3E0F55DAE5CAFC0
:105C92005D745E12727574058E048F05FF12726553
:105CA200AE5AAF5BED2FFFEC3EFE8E5C8F5D900037
:105CB2003CE0FCA3E0FDEF2DFDEE3CFC8C5C8D5D39
:105CC200123E6F75A7009000F6E0B40103123EA5E4
:105CD2008019123D75123E2B123DB4123E6F75A70C
:105CE200009000F6E0B40103123EA58043123D7518
:105CF200123E2B9000D8E0B4031275A710123E6F2B
:105D02009000F6E0B40103123EA5802175A7109021
:105D120000F6E0B40106A203B3B340028005123ECE
:105D22006F800A9000F6E0B40203123E6F75A7007E
:105D3200D20CD20DC20ED20FA20FB3B350089000F4
:105D420055E0655F6003025EC3A202B35006A20182
:105D5200B3B34003025EBB9000D8E0B404028003F8
:105D6200025E789008FAE0B402028003025E5DA24D
:105D720020B3406D123D75900129E0D39403401F7A
:105D820090001CE0FEA3E0FF900124E01272757403
:105D9200C88E048F05FF1272658C5C8D5D800A903F
:105DA200001CE0F55CA3E0F55DAE5CAF5D745E12D5
:105DB200727574058E048F05FF127265AE5AAF5B61
:105DC200ED2FFFEC3EFE8E5C8F5D90003CE0FCA36D
:105DD200E0FDEF2DFDEE3CFC8C5C8D5D123E3680CD
:105DE2006E123DB4900129E0D39407401F90001C2D
:105DF200E0FEA3E0FF900128E012727574C88E04E1
:105E02008F05FF1272658C5C8D5D800A90001CE02C
:105E1200F55CA3E0F55DAE5CAF5D745E1272757405
:105E2200058E048F05FF127265AE5AAF5BED2FFF30
:105E3200EC3EFE8E5C8F5D90003CE0FCA3E0FDEF4B
:105E42002DFDEE3CFC8C5C8D5D123E8A75A70090A8
:105E520000F6E0B40103123EA58019123D75123E10
:105E620036123DB4123E8A75A7009000F6E0B401E6
:105E720003123EA58043123D75123E369000D8E0D3
:105E8200B4031275A710123E8A9000F6E0B4010323
:105E9200123EA5802175A7109000F6E0B40106A27B
:105EA20003B3B340028005123E8A800A9000F6E0F6
:105EB200B40203123E8A75A700D20CD20DD20EC2D2
:0E5EC2000FE571906B96F82828739000FDE0B4
:036B9600025ECCD0
:105ED000906BC9F828287312260C801212260C80A9
:0E5EE0000D12269680081227428003122742D8
:0F6BC900025ED7025EDC025EE1025EE6025EEB78
:105EEE007571010263E912286E122985757102021D
:105EFE0063E9122D21A204B340139000E2E075F085
:105F0E001DA4FFAEF0900018EEF0A3EFF0900890F5
:105F1E00E0FEA3E0FF740A127275900012E0FCA37B
:105F2E00E0FD74098F02FF1272658D078C038E04DB
:105F3E008A058B06127163900894EEF0A3EFF0744D
:105F4E0078BE00039F500B7478900894F8E4F0E844
:105F5E00A3F0E5377003753701900894E0FEA3E0D7
:105F6E00FFE5372FFF50010E900894EEF0A3EFF0EF
:0B5F7E00757103A230401F900060E02E
:066B9900025EF4025F0041
:105F8900906BD8F8282873801275710A800D757185
:0B5F99000B800875710C800375710D02
:0F6BD800025F90025F92025F97025F9C025FA1D3
:105FA4000263E99006D7E06006750801122E4FA23D
:105FB40032B3401675E70090078EE0B42906E5B5C4
:105FC4004408F5B575E71002606F9000CBE0D394F8
:105FD40002404590009FE02403A852B80004955362
:105FE40050099000A1E0D395625002800ED202A223
:105FF400284006740890005FF0D22890009FE0A823
:1060040052B80005D39553500B9000A1E02403C36C
:1060140095625002C202805390009FE02403A8526C
:10602400B8000495535010E560C395615009900081
:10603400A1E0D395625002800ED202A228400674D9
:106044000890005FF0D22890009FE0A852B80005A5
:10605400D395535014E561240FC39560400B900011
:10606400A1E02403C395625002C202A2024002C20C
:1060740028A232B35005A202B34002801375E70090
:1060840090078EE0B42906E5B554F7F5B575E71029
:106094009000E5E07007E56BC3941440028002D2DF
:1060A400029000DAE0B40102D202A2024005757146
:1060B40004800A75711090001EE4F0A3F00263E9F5
:0460C4009000CBE09D
:066B9F00025FA70260C4C2
:1060C800906BE7F8282873121397801212139780A1
:0E60D8000D12154A80081216018003121601DF
:0F6BE7000260CF0260D40260D90260DE0260E378
:1060E6007571050263E912175A7571069006DFE0AD
:1060F6006006750803122E4F9006E3E060067508E9
:1061060004122E4F0263E990005AE06006A204B31F
:10611600B34002800DE55FD39409500690005AE023
:1061260014F01219E37571079006E7E0600675082A
:1061360005122E4F9006EBE06006750806122E4FEC
:106146000263E9900118E0B40203121308121E4B11
:106156007571089006EFE06006750807122E4F90DD
:1061660006F3E06006750808122E4F0263E9121F57
:106176002D7571090263E9122305A20CB35005A21D
:106186000DB340028008D20CD20DD20ED20F75711B
:10619600109006F7E06006750809122E4F9006FB70
:1061A600E0600675080A122E4F0263E9900040E08F
:1061B600C394465008C2967446900040F09000562C
:1061C600E0B4011DE537240AF537900894E0FEA3F4
:1061D600E0FF740A2FFF50010E900894EEF0A3EF33
:1061E600F085375B755A0090004EE0F57412401F3B
:1061F600E55D900040F0900008E55AF0A3E55BF0FD
:10620600E574900041F0C211900894E0F55AA3E0BD
:10621600F55B90004EE0F57412401FE55D90003E80
:10622600F0900000E55AF0A3E55BF0E57490003FBE
:10623600F0C2107571030263E9900044E0C394460E
:106246005008C2957446900044F0900057E0B4019F
:106256001DE537240AF537900894E0FEA3E0FF74A5
:106266000A2FFF50010E900894EEF0A3EFF0853749
:106276005B755A0090004FE0F57412401FE55D9083
:106286000044F090000AE55AF0A3E55BF0E574904F
:106296000045F0C213900894E0F55AA3E0F55B9030
:1062A600004FE0F57412401FE55D900042F090004B
:1062B60002E55AF0A3E55BF0E574900043F0C212E4
:1062C6007571030263E9900048E0C394465008C222
:1062D600967446900048F0900058E0B4011DE537EA
:1062E600240AF537900894E0FEA3E0FF740A2FFF16
:1062F60050010E900894EEF0A3EFF085375B755AC7
:1063060000900050E0F57412401FE55D900048F0E3
:1063160090000CE55AF0A3E55BF0E574900049F0B7
:10632600C215900894E0F55AA3E0F55B900050E0A2
:10633600F57412401FE55D900046F0900004E55AA2
:10634600F0A3E55BF0E574900047F0C214757103A5
:106356000263E990004CE0C394465008C295744627
:1063660090004CF0900059E0B4011DE537240AF581
:1063760037900894E0FEA3E0FF740A2FFF50010E49
:10638600900894EEF0A3EFF085375B755A00900005
:1063960051E0F57412401FE55D90004CF090000E40
:1063A600E55AF0A3E55BF0E57490004DF0C2179056
:1063B6000894E0F55AA3E0F55B900051E0F57412FD
:1063C600401FE55D90004AF0900006E55AF0A3E50F
:1063D6005BF0E57490004BF0C21675710380048083
:0363E60002800032
:106BA5000260EC02610D02614902617402617D02BD
:106BB50061B202623F0262CC0263590263E502637D
:046BC500E70263E997
:1063E90090003EE0B55F73A210404F900000E0FEC0
:1063F900A3E0FFEF4E6021AE56AF57900000E0FCDE
:10640900A3E0FD120003740A8E048F05FF12726562
:10641900900000ECF0A3EDF090003FE0601A9000CE
:1064290000E0FEA3E0FFAC56AD57EF2DFDEE3CFCBE
:10643900900000ECF0A3EDF0D210AE54AF559000EF
:1064490000E0FCA3E0FDEFC39DEE9C400D124AF96C
:10645900D296C21074C890003EF0A210B3B3500790
:1064690090003EE0B55F02800D124AF9D29674C8D9
:1064790090003EF0C210900040E0B55F70A211405C
:106489004F900008E0FEA3E0FFEF4E6021AE56AF4B
:1064990057900008E0FCA3E0FD120003740A8E0483
:1064A9008F05FF127265900008ECF0A3EDF09000E3
:1064B90041E0601A900008E0FEA3E0FFAC56AD573A
:1064C900EF2DFDEE3CFC900008ECF0A3EDF0D211AD
:1064D900AE54AF55900008E0FCA3E0FDEFC39DEE7C
:1064E9009C400AC2967446900040F0C211A211B3B2
:1064F900B35007900040E0B55F02800AC296744627
:10650900900040F0C211900042E0B55F73A21240C2
:106519004F900002E0FEA3E0FFEF4E6021AE56AFC0
:1065290057900002E0FCA3E0FD120003740A8E04F8
:106539008F05FF127265900002ECF0A3EDF0900058
:1065490043E0601A900002E0FEA3E0FFAC56AD57AD
:10655900EF2DFDEE3CFC900002ECF0A3EDF0D21221
:10656900AE54AF55900002E0FCA3E0FDEFC39DEEF1
:106579009C400D124AF9D295C21274C8900042F09B
:10658900A212B3B35007900042E0B55F02800D122A
:106599004AF9D29574C8900042F0C212900044E0C2
:1065A900B55F70A213404F90000AE0FEA3E0FFEF31
:1065B9004E6021AE56AF5790000AE0FCA3E0FD12F1
:1065C9000003740A8E048F05FF12726590000AECAD
:1065D900F0A3EDF0900045E0601A90000AE0FEA3F8
:1065E900E0FFAC56AD57EF2DFDEE3CFC90000AECF8
:1065F900F0A3EDF0D213AE54AF5590000AE0FCA31E
:10660900E0FDEFC39DEE9C400AC29574469000449C
:10661900F0C213A213B3B35007900044E0B55F0270
:10662900800AC2957446900044F0C213900046E077
:10663900B55F73A214404F900004E0FEA3E0FFEFA2
:106649004E6021AE56AF57900004E0FCA3E0FD1266
:106659000003740A8E048F05FF127265900004EC22
:10666900F0A3EDF0900047E0601A900004E0FEA36B
:10667900E0FFAC56AD57EF2DFDEE3CFC900004EC6D
:10668900F0A3EDF0D214AE54AF55900004E0FCA392
:10669900E0FDEFC39DEE9C400D124AF9D296C2145B
:1066A90074C8900046F0A214B3B35007900046E0B6
:1066B900B55F02800D124AF9D29674C8900046F06F
:1066C900C214900048E0B55F70A215404F90000CCD
:1066D900E0FEA3E0FFEF4E6021AE56AF5790000CED
:1066E900E0FCA3E0FD120003740A8E048F05FF127B
:1066F900726590000CECF0A3EDF0900049E0601A8F
:1067090090000CE0FEA3E0FFAC56AD57EF2DFDEE77
:106719003CFC90000CECF0A3EDF0D215AE54AF5553
:1067290090000CE0FCA3E0FDEFC39DEE9C400AC283
:10673900967446900048F0C215A215B3B35007905D
:106749000048E0B55F02800AC2967446900048F09E
:10675900C21590004AE0B55F73A216404F9000063B
:10676900E0FEA3E0FFEF4E6021AE56AF5790000662
:10677900E0FCA3E0FD120003740A8E048F05FF12EA
:106789007265900006ECF0A3EDF090004BE0601A02
:10679900900006E0FEA3E0FFAC56AD57EF2DFDEEED
:1067A9003CFC900006ECF0A3EDF0D216AE54AF55C8
:1067B900900006E0FCA3E0FDEFC39DEE9C400D12A6
:1067C9004AF9D295C21674C890004AF0A216B3B31A
:1067D900500790004AE0B55F02800D124AF9D29540
:1067E90074C890004AF0C21690004CE0B55F70A2E0
:1067F90017404F90000EE0FEA3E0FFEF4E6021AE80
:1068090056AF5790000EE0FCA3E0FD120003740A96
:106819008E048F05FF12726590000EECF0A3EDF067
:1068290090004DE0601A90000EE0FEA3E0FFAC5628
:10683900AD57EF2DFDEE3CFC90000EECF0A3EDF012
:10684900D217AE54AF5590000EE0FCA3E0FDEFC3A4
:106859009DEE9C400AC295744690004CF0C217A266
:1068690017B3B3500790004CE0B55F02800AC29598
:10687900744690004CF0C2179000E8E0B402028020
:106889000302699A90007FE0D39567506490007F76
:10689900E0F4042567FE9000EBE08E00F5F0E88453
:1068A900FF7E008F74EFC39410500CEF8574F0A431
:1068B900FDACF08D7480037574FF90007FE0D39573
:1068C90074400B90007FE0C39574F5728003757274
:1068D90000900106E0D395724006900106E0F5723A
:1068E900900107E0C395725006900107E0F57280A8
:1068F9007190007FE0C39567FE9000EBE08E00F594
:10690900F0E884FF7E008F74EFC39410500CEF857C
:1069190074F0A4FDACF08D7480037574FF85745B0D
:10692900755A0090007FE0255BFFAE5A50010E8E2C
:106939005A8F5B74FFBE0009D39F4005855B728047
:10694900037572FF900106E0D39572400690010627
:10695900E0F572900107E0C395725006900107E0D7
:10696900F572A204B3B3500D900080E0FE9000F3DD
:10697900E0D39E5002800A740790005FF0C29780AE
:106989001075A710E5CDC395724004C2978002D255
:1069990097E570C39413501DE57075F00284AFF04C
:1069A9007E00EF4E70051232FC800AA2EDB340055D
:1069B900C2ED1232FCAE54AF557410C39F74279EBA
:1069C900400C90007EE0C3945A4003026B3CA2093C
:1069D900B340091246BF740690005FF0A20BB35092
:1069E9000EE562D394334007E562C394CC4002803C
:1069F90041900118E0B40214121281900082E075EE
:106A0900F05EA4FFAEF08E5C8F5D800F900094E085
:106A190075F05EA4FFAEF08E5C8F5DE55D455C6050
:106A290011E5B54401F5B5742B90007DF0124A4289
:106A3900D20B90007EE0D394014007E562C3941A1B
:106A490040028002C20B9006D7E060067508011269
:106A59002E4F9006DFE06006750803122E4F900650
:106A6900E3E06006750804122E4F9006E7E0600621
:106A7900750805122E4F9006EBE0600675080612A0
:106A89002E4F9006EFE06006750807122E4F90060C
:106A9900F3E06006750808122E4F9006F7E06006CD
:106AA900750809122E4F9006FBE0600675080A1258
:106AB9002E4F90007EE0C3945A5010E570B413092C
:106AC90090007EE004F0757000803FE570B4130318
:106AD900757000C28E758D00758B007565007555D2
:106AE90001755400D28E90007DE0C3944150089006
:106AF900007DE004F08006744190007DF090007DF7
:106B0900E0B44106E5B554FEF5B590007EE0D394B6
:106B1900014007E56BC3944140028006740E900062
:106B29005FF09008A7E06006900115E0600280031D
:066B3900120BD7024FEE23
:106BF6000000010001400160018001A001C001E028
:106C060002000300039603B603D603F4040005004E
:106C16000512052405360548055A056C057E0590BE
:106C260005A805C005DE0600061406280646066EFB
:106C360006AE05CF06EE00FF013F015F017F019F13
:106C460001BF01DF01FF02FF039503B503D503F37F
:106C560003FF04FF05110523053505470559056B97
:106C6600057D058F05A705BF05CE05F10613062789
:106C76000645066D06AD06ED05DD06FF0FAA0FA556
:106C86000F9F0F9A0F940F8D0F870F800F780F713C
:106C96000F680F600F570F4E0F450F3B0F300F2534
:106CA6000F1A0F0E0F020EF50EE80EDB0ECC0EBEFF
:106CB6000EAE0E9F0E8E0E7D0E6C0E5A0E470E34C5
:106CC6000E200E0C0DF70DE20DCB0DB50D9D0D85AD
:106CD6000D6D0D540D3A0D200D050CE90CCE0CB1C1
:106CE6000C940C760C580C3A0C1B0BFB0BDB0BBBF9
:106CF6000B9A0B790B570B350B130AF10ACE0AAB1D
:106D06000A870A640A400A1C09F809D409B0098CE2
:106D160009670943091F08FB08D608B2088E086AE6
:106D26000846082307FF07DC07B9079607730751CC
:106D3600072F070D06EC06CA06AA06890669064944
:106D4600062A060A05EC05CD05B005920575055817
:106D5600053C0520050504EA04CF04B5049C04821D
:106D66000469045104390422040B03F403DE03C846
:106D760003B2039D038903750361034D033B032897
:106D86000316030402F202E102D102C002B002A01D
:106D9600029102820273026502570249023C022FE7
:106DA60002220216020901FD01F201E601DB01D011
:106DB60001C601BB01B101A7019D0194018B0182AE
:106DC60001790170016801600158015001480141D3
:106DD60001390132012B0125011E01180111010B98
:106DE600010500FF00FA0FA60FA00F990F920F8B57
:106DF6000F840F7C0F740F6B0F620F580F4E0F43EB
:106E06000F380F2C0F1F0F120F050EF70EE80ED8B6
:106E16000EC80EB70EA50E930E800E6C0E580E42BF
:106E26000E2C0E150DFD0DE40DCB0DB10D950D7946
:106E36000D5D0D3F0D200D010CE10CC00C9E0C7C70
:106E46000C590C350C100BEA0BC40B9E0B760B4F32
:106E56000B260AFD0AD40AAA0A800A550A2A09FF3D
:106E660009D409A8097C0950092508F908CD08A103
:106E76000875084A081E07F307C8079D07730749E0
:106E8600072006F706CE06A6067E06570630060A31
:106E960005E405BF059B057705540532051004EF8B
:106EA60004CE04AE048F047104530435041903FDA3
:106EB60003E203C703AD0394037B0363034B03346D
:106EC600031E030802F302DE02CA02B602A30291FF
:106ED600027F026D025C024C023C022C021D020E75
:106EE600020001F201E401D701CA01BE01B101A607
:106EF600019A018F0185017A01700166015D0153D6
:106F0600014A014101390131012901210119011209
:106F1600010B010400FD00F700F000EA00E400DECA
:106F260000D900D300CE00C900C400BF00BA00B526
:106F360000B100AD00A800A400A0009C0099009537
:106F46000091008E008A008700840081007E007B0D
:10009E0075B50075840175A70075FFA075EF069004
:1000AE00005BE4F075C91075A70F75A1C775A700A1
:1000BE0075D90075CE0C75A70F75F1FE75F2FF752B
:1000CE00F30775F47875A4BA75A5FF75A60775AE16
:1000DE000075AFFF75D48175D5FF75D6FF75D7FF47
:1000EE0075A70075A20175A14775F8092275E60876
:1000FE0075E71075BC0175BE0475BD6C75BE0775D0
:10010E00BDA075BE0875BD0175BC0075BB1875BC6C
:10011E002075BA0875E88075D11375A70F75E105BE
:10012E0075E20075C7401246BF75970075978074CB
:10013E000A1272557597C0E5975420700280F875B3
:10014E008F0275A700D2AF75980075A90C75A70F11
:10015E0075AB4375ADFB75AC1E75A71075C91875DB
:10016E00CA0075CB0075C80475A700758912758E07
:10017E0004758C00758A00C2A9D28C758D00758BA2
:10018E0000D2ABD28E75B62075D944C2992290009A
:10019E0092E09008A6F090009DE09008A7F09000E5
:1001AE009EE09008A8F09000BDE09008A9F09000A5
:1001BE00CAE09008AAF09000D8E09008ABF090004A
:1001CE00E6E09008ACF09000E8E09008ADF090000A
:1001DE00F6E09008AEF0900103E09008AFF09001C9
:1001EE0004E09008B0F0900116E09008B1F0900194
:1001FE002EE09008B3F090017CE09008B4F09001EE
:10020E007DE09008B5F090017EE09008B6F0900188
:10021E0015E09008B7F09000FFE09008B8F090005D
:10022E00B6E09008B9F09000B7E09008BAF09000F0
:10023E00B1E09008BBF09000B2E09008BCF09001E5
:10024E001BE09008BDF090011CE09008BEF09001FC
:10025E001DE09008BFF090011EE09008C0F09001E4
:10026E001FE09008C1F09006D6E09008C2F090060C
:10027E00DAE09008C3F09006DEE09008C4F0900635
:10028E00E2E09008C5F09006E6E09008C6F0900611
:10029E00EAE09008C7F09006EEE09008C8F09006ED
:1002AE00F2E09008C9F09006F6E09008CAF09006C9
:1002BE00FAE09008CBF090077EE09008CCF0900723
:1002CE007FE09008CDF0900780E09008CEF0900788
:1002DE0081E09008CFF0900782E09008D0F0900770
:1002EE0083E09008D1F0900784E09008D2F0900758
:1002FE0085E09008D3F0900786E09008D4F0900740
:10030E0087E09008D5F0900788E09008D6F0900727
:10031E0089E09008D7F090078AE09008D8F090070F
:10032E008BE09008D9F090078CE09008DAF09007F7
:10033E008DE09008DBF090078EE09008DCF09001E5
:10034E0020E09008DDF0900121E09008DEF09001B1
:10035E0022E09008DFF0900123E09008E0F0900199
:10036E0024E09008E1F0900125E09008E2F0900181
:10037E0026E09008E3F0900127E09008E4F0900169
:10038E0028E09008E5F0900129E09008E6F0900052
:10039E00C4E09008E7F09000FCE09008E8F09001CF
:1003AE0034E09008E9F0900135E09008EAF02290F0
:1003BE0008A6E0900092F09008A7E090009DF090C3
:1003CE0008A8E090009EF09008A9E09000BDF09083
:1003DE0008AAE09000CAF09008ABE09000D8F09028
:1003EE0008ACE09000E6F09008ADE09000E8F090E8
:1003FE0008AEE09000F6F09008AFE0900103F090A8
:10040E0008B0E0900104F09008B1E0900116F09071
:10041E0008B3E090012EF09008B7E0900115F0902F
:10042E0008B8E09000FFF09008B9E09000B6F090A8
:10043E0008BAE09000B7F09008BBE09000B1F090E1
:10044E0008BCE09000B2F09008BDE090011BF09067
:10045E0008BEE090011CF09008BFE090011DF090E6
:10046E0008C0E090011EF09008C1E090011FF090CE
:10047E0008C2E09006D6F09008C3E09006DAF0903D
:10048E0008C4E09006DEF09008C5E09006E2F09019
:10049E0008C6E09006E6F09008C7E09006EAF090F5
:1004AE0008C8E09006EEF09008C9E09006F2F090D1
:1004BE0008CAE09006F6F09008CBE09006FAF090AD
:1004CE0008CCE090077EF09008CDE090077FF0908A
:1004DE0008CEE0900780F09008CFE0900781F09072
:1004EE0008D0E0900782F09008D1E0900783F0905A
:1004FE0008D2E0900784F09008D3E0900785F09042
:10050E0008D4E0900786F09008D5E0900787F09029
:10051E0008D6E0900788F09008D7E0900789F09011
:10052E0008D8E090078AF09008D9E090078BF090F9
:10053E0008DAE090078CF09008DBE090078DF090E1
:10054E0008DCE090078EF09008DDE0900120F0903E
:10055E0008DEE0900121F09008DFE0900122F0909B
:10056E0008E0E0900123F09008E1E0900124F09083
:10057E0008E2E0900125F09008E3E0900126F0906B
:10058E0008E4E0900127F09008E5E0900128F09053
:10059E0008E6E0900129F09008E7E09000C4F090A2
:1005AE0008E8E09000FCF09008E9E0900134F0904B
:1005BE0008EAE0900135F02275480090089EE4F0BC
:1005CE00A3F0753200753100754E00754F00C22CC8
:1005DE00D22D9008A7E06002D22474FE9008A0F8F5
:1005EE00E4F0E8A3F074FE9008A4F8E4F0E8A3F0B9
:1005FE0074FE9008A2F8E4F0E8A3F0745A9008F89C
:10060E00F0745A9008F9F0D22EC22AC230C22FC20C
:10061E002BC232C23822750B00750A00AE0AAF0B20
:10062E00AC08AD09EDC39FEC9E401674FF127255D7
:10063E0075CF01780B740126F6500418E436F65087
:10064E00DB22C2AF75D904758F0375B7A575B7F1E7
:10065E0090F800E4F0758F0175B7A575B7F1E52830
:10066E0090F800F075B7A575B7F190F801E4F07544
:10067E00B7A575B7F19008ECE090F802F075B7A544
:10068E0075B7F19008F0E090F803F075B7A575B75F
:10069E00F19008EDE090F804F075B7A575B7F190FC
:1006AE0008EEE090F805F075B7A575B7F19008EF74
:1006BE00E090F806F075B7A575B7F19008F1E090E7
:1006CE00F807F0758F0075D944D2AF2290005BE029
:1006DE00B4AB61C2AF75D90475B62275F522758FAC
:1006EE000375B7A575B7F1740090F600F0758F011C
:1006FE00755B00755A00AE5AAF5B7445BE00279FFE
:10070E00402475B7A575B7F19008A6120048E0FC15
:10071E0090F600120048ECF0785B740126F6500457
:10072E0018E436F650D0758F0075F51175B6207534
:10073E00D944D2AF22C2AF75F52275D904755B00CC
:10074E00755A00AE5AAF5B7445BE00229F401F9093
:10075E00F600120048E493FC9008A6120048ECF054
:10076E00785B740126F6500418E436F650D575D928
:10077E004475F511D2AF2290005BE0B4AA0280035B
:10078E000208C2C2AF75D90475B62275F522758FEF
:10079E000375B7A575B7F1740090F400F075B7A5A1
:1007AE0075B7F1740090F200F075B7A575B7F174D6
:1007BE000090F000F075B7A575B7F1740090EE00DB
:1007CE00F0758F01755B00755A00AE5AAF5B74FF02
:1007DE00C39F74019E402475B7A575B7F190009024
:1007EE00120048E0FC90F400120048ECF0785B74C4
:1007FE000126F6500418E436F650CF755B00755A94
:10080E0000AE5AAF5B74FFC39F74019E402475B750
:10081E00A575B7F1900290120048E0FC90F200121C
:10082E000048ECF0785B740126F6500418E436F6B6
:10083E0050CF755B00755A00AE5AAF5B74FFC39F05
:10084E0074019E402475B7A575B7F19004901200FF
:10085E0048E0FC90F000120048ECF0785B74012642
:10086E00F6500418E436F650CF755B00755A00AE9C
:10087E005AAF5B74FFC39F74019E402475B7A57574
:10088E00B7F1900690120048E0FC90EE001200487E
:10089E00ECF0785B740126F6500418E436F650CF6F
:1008AE00758F0075F51175B62075D944D2AF743AAF
:1008BE00900790F02290005BE0B4AA028003020A37
:1008CE0000C2AF75D90475B62275F522758F037502
:1008DE00B7A575B7F1740090EC00F075B7A575B7B4
:1008EE00F1740090EA00F075B7A575B7F174009039
:1008FE00E800F075B7A575B7F1740090E600F075D5
:10090E008F01755B00755A00AE5AAF5B74FFC39FC3
:10091E0074019E402475B7A575B7F1900090120032
:10092E0048E0FC90EC00120048ECF0785B74012675
:10093E00F6500418E436F650CF755B00755A00AECB
:10094E005AAF5B74FFC39F74019E402475B7A575A3
:10095E00B7F1900290120048E0FC90EA00120048B5
:10096E00ECF0785B740126F6500418E436F650CF9E
:10097E00755B00755A00AE5AAF5B74FFC39F74016E
:10098E009E402475B7A575B7F1900490120048E00B
:10099E00FC90E800120048ECF0785B740126F650EB
:1009AE000418E436F650CF755B00755A00AE5AAF98
:1009BE005B74FFC39F74019E402475B7A575B7F194
:1009CE00900690120048E0FC90E600120048ECF011
:1009DE00785B740126F6500418E436F650CF758F06
:1009EE000075F51175B62075D944D2AF743A9007DB
:1009FE0090F022C2AF75D90475F522755B00755A59
:100A0E0000AE5AAF5B74FFC39F74019E401F90F4FB
:100A1E0000120048E493FC900090120048ECF0782D
:100A2E005B740126F6500418E436F650D4755B005C
:100A3E00755A00AE5AAF5B74FFC39F74019E401F80
:100A4E0090F200120048E493FC900290120048ECE1
:100A5E00F0785B740126F6500418E436F650D4751F
:100A6E005B00755A00AE5AAF5B74FFC39F74019E54
:100A7E00401F90F000120048E493FC900490120086
:100A8E0048ECF0785B740126F6500418E436F65004
:100A9E00D4755B00755A00AE5AAF5B74FFC39F747A
:100AAE00019E401F90EE00120048E493FC900690C9
:100ABE00120048ECF0785B740126F6500418E43608
:100ACE00F650D475F51175D944D2AF74019000D992
:100ADE00F0743A900790F09008FF7401F022C2AFC4
:100AEE0075D90475F522755B00755A00AE5AAF5B69
:100AFE0074FFC39F74019E401F90EC00120048E4E7
:100B0E0093FC900090120048ECF0785B740126F68E
:100B1E00500418E436F650D4755B00755A00AE5A80
:100B2E00AF5B74FFC39F74019E401F90EA001200DA
:100B3E0048E493FC900290120048ECF0785B74014C
:100B4E0026F6500418E436F650D4755B00755A003C
:100B5E00AE5AAF5B74FFC39F74019E401F90E800B6
:100B6E00120048E493FC900490120048ECF0785B7D
:100B7E00740126F6500418E436F650D4755B0075F1
:100B8E005A00AE5AAF5B74FFC39F74019E401F9014
:100B9E00E600120048E493FC900690120048ECF038
:100BAE00785B740126F6500418E436F650D475F5C9
:100BBE001175D944D2AF74029000D9F0743A9007EF
:100BCE0090F074029008FFF02274019000D9F0901A
:100BDE0008A7E0903CBBF828287380188016A2A3C3
:100BEE00400674029000D9F0800AA2A44006740256
:040BFE009000D9F09A
:0C3CBB00020BE8020BEA020BEC020BF813
:100C02009000D9E0B40105A236B34002801AD23670
:100C12001246BF120A0174019000D9F01203BD12EC
:100C22003F5F741B90005FF09000D9E0B40206A20F
:100C320036B3B34002801AC2361246BF120AEC74AF
:100C4200029000D9F01203BD123F5F741B90005F47
:100C5200F022E54F64046006E59964FF600280318A
:100C6200A22C4004D22C8027E54F600874E6254F61
:100C720090005FF0E54E600874F0254E90005FF042
:100C8200E54FB4010280FE754F00754E00C22C8004
:100C920002C22CE54F903CC7F8282873754F00E537
:100CA20099B4FF03754E01E599B4FE03754E02E552
:100CB20099B4FD03754E03E599B4FC03754E04E542
:100CC20099B4FA03754E05E599B4FB06754F011206
:100CD20046BFE599B4F906754F041246BFE599B4CB
:100CE200F7331246BFC29C74AB90005BF01206DA77
:100CF20074AA90005BF09008FFE0B401051207852A
:100D020080031208C390005BE4F0D29C754F00751B
:100D12004E007599F7E599D394E54007E599C39498
:100D2200F040028016859950754F027E017F00E5E2
:100D320050C394E61272758E338F3490089EE4F09D
:100D4200A3F0E599D394C24007E599C394E6400223
:100D52008028859950754F0374E5C39550F5347515
:100D62003300AE33AF34906BF6127244E493F874EE
:100D7200019390089EC8F0A3C8F0D2990210DF90A8
:100D820008B3E0700AA225B35005A226B340028040
:100D92005C90089EE0FEA3E0FF74FFBE00039F503C
:100DA20009EFC39446EE9406402B90089EE0FEA302
:100DB200E0FFEFD3946DEE94064009EFC394EEEE9C
:100DC2009406401190089EE0FEA3E0FFEFD394FF4B
:100DD200EE9406401390089EE0FEA3E0FF90009080
:100DE200120048E599F08003859975801190089E5C
:100DF200E0FEA3E0FF900090120048E599F0900811
:100E02009E12728390089EE0FEA3E0FFEFB40106FB
:100E1200EEB407028003020EDA900790E0B43C02BF
:100E22008003020EDAA225B35005A226B340028047
:100E320055C29C1203BD90009DE09008FEF0124046
:100E4200A190017CE09008B4F090017DE09008B59B
:100E5200F090017EE09008B6F074AB90005BF01267
:100E620006DA74AA90005BF09008FFE0B401051264
:100E7200078580031208C39008FFE09000D9F09024
:100E8200005BE4F08047C29C12019C74009008B49D
:100E9200F074009008B5F074009008B6F090009DD0
:100EA200E09008FEF01240A174AB90005BF01206D5
:100EB200DA74AA90005BF01207851208C3D29C75FF
:100EC20099FB75096475080012062480FED29C7590
:100ED2004F00754E007599FB0210DF90089EE0FEF0
:100EE200A3E0FFEF4E700685993275310090089E9F
:100EF200E0FEA3E0FF74016F4E701BAC31AD32AA6D
:100F020033AB34ED2BFBEC3AFA8A068B0790009058
:100F1200120048E599F090089E12728390089EE0B4
:100F2200FEA3E0FF74026F4E7021AC31AD327456F5
:100F32006D4C7006E55064E6600280031246BF12F3
:100F420040A1855099754F00754E000210DF900840
:100F52009EE0FEA3E0FF900090120048E599F09019
:100F6200089E12728390089EE0FEA3E0FFAC33ADB0
:100F7200348F028E038C068D07906C3C127244E40F
:100F820093F9740193FEEAD39EEB99400985509937
:100F9200754F00754E000210DF90089EE0FEA3E040
:100FA200FF900090120048E599F090089E1272831B
:100FB20090089EE0FEA3E0FFEFB40006EEB401024B
:100FC20080030210DF900071E0D394C7400B9000C1
:100FD20071E0C394C8F551801A900071E0D3946314
:100FE200400B900071E0C39464F55180069000714B
:100FF200E0F551E55175F002A4FFAEF08F74EF9069
:1010020000901272A6EFFCE0FDEC9000931272A623
:10101200EDFCE0FDEC2DB5510280030210D10FEF83
:101022009000901272A6E574FFE0FCEF900094121B
:1010320072A6ECFFE0FCEFC39CB5510280030210E4
:10104200D1E5749000921272A6E574FFE0FCEF9075
:1010520000951272A6ECFFE0FCEF2CB55171E5741D
:101062009000961272A6E0C395519008ECF0E574D8
:101072009000971272A6E0C395519008EDF0E574C6
:1010820090009A1272A6E0C395519008EEF0E574B2
:1010920090009B1272A6E0C395519008EFF0E574A0
:1010A20090009C1272A6E0C395519008F0F0E5748E
:1010B20090009D1272A6E0C395519008F1F01206BD
:1010C200507599F975096475080012062480FE7539
:0D10D20099FF75096475080012062480FE60
:0F3CC700020C9E020D81020EDD020F50020F9BB8
:1010DF0022E54E903CD6F82828730211C490089E42
:1010EF00E0FEA3E0FF900061120048E0F599900840
:1010FF009E12728390089EE0FEA3E0FF741C6F4E59
:10110F007003754E000211C4856F990211C49008C7
:10111F009EE0FEA3E0FF900090120048E0F599EFEB
:10112F00B40107EEB40703754E0090089E12728348
:07113F000211C490089FE0BB
:0F3CD6000210E90210EC02111702111D02114237
:10114600903D48F828287385539980678560998073
:1011560062856299805D8566998058856899805315
:10116600856999804E856A998049856B99804490F6
:10117600001FE0F599803CA22DB340077599FAC28D
:101186002D8017A224B3400575990F800B90005F40
:10119600E0F59990005FE4F0C2248017856C998091
:1011A60012856799800D856D9980087599FC800375
:0311B600754E0073
:103D480002114D02115202115702115C0211610257
:103D5800116602116B02117002117502117D0211B8
:0D3D6800A20211A70211AC0211B10211B6A6
:0B11B90090089E1272838003123FBA60
:033CE5000211C108
:1011C40022E538255BFFAE5A50010E9000901200C4
:1011D40048E0F539E538255BFFAE5A50010E0FBFE4
:1011E40000010E900090120048E0F53A85403CE57D
:1011F40039B53A058539388041E53AD39539401DEA
:10120400E53AC39539853BF0A4FFAEF0E53C8E0486
:101214008F05FF127265ED2539F538801DE539C358
:10122400953A853BF0A4FFAEF0E53C8E048F05FFB4
:10123400127265EDF4042539F53822E53AD395396F
:10124400401DE53AC39539853BF0A4FFAEF0E53C7B
:101254008E048F05FF127265ED2539F538801DE582
:1012640039C3953A853BF0A4FFAEF0E53C8E048F7C
:1012740005FF127265EDF4042539F53822900096C5
:10128400E0B4017FE56875F00A84FF7E008F38E5DD
:101294006875F00A84ADF07C008D3B75400A755A80
:1012A40005755B24E538C3941150051211C58006F9
:1012B4009005C5E0F538E538C394F05008E538905A
:1012C4000082F0800674EF900082F0E56875F00A01
:1012D40084FF7E008F38E56875F00A84ADF07C00E9
:1012E4008D3B75400A755A05755B5AE538C39411F0
:1012F40050051211C580069005FBE0F538E53890DD
:10130400005AF022900096E0B40102800302139682
:10131400E56875F00A84FF7E008F38E56875F00A89
:1013240084ADF07C008D3B75400A755A05755B36BB
:10133400E538C3941150051211C580069005D7E015
:10134400F538E538C394F0500585384C8003754C66
:10135400EFE56875F00A84FF7E008F38E56875F064
:101364000A84ADF07C008D3B75400A755A05755BA7
:1013740048E538C3941150051211C580069005E95B
:10138400E0F538E538C394F0500585384D80037591
:101394004DEF22E56075F00484FF7E008F38E56030
:1013A40075F00484ADF07C008D3B754004755A01E2
:1013B400755B00E538C3943F50051211C580069053
:1013C40001CFE0F538E538900898F8E4F0E8A3F0A8
:1013D40090005EE075F020A4FFAEF09000E1E08E96
:1013E400048F05FF1272658D389000C9E0D39560B3
:1013F40050030214A29000EDE0D395604010ED90EC
:1014040001D01272A6E0F52C752B0002149F9000F7
:10141400B8E0D395604043E5389001D01272A6E05D
:10142400F539E5389001F01272A6E0F53A9000ED36
:10143400E0F4042560F53B9000B8E0FE9000EDE098
:10144400F4042EF53CE539B53A05853938800312A4
:10145400123F85382C752B008041E5389001F0123D
:1014640072A6E0F539E5389002101272A6E0F53A5A
:101474009000B8E0F4042560F53B9000C9E0FE90CC
:1014840000B8E0F4042EF53CE539B53A0585393861
:10149400800312123F85382C752B000215499000E9
:1014A400F0E0D395605011E5389002501272A6E036
:1014B400F52C752B000215499000B9E0D3956050C6
:1014C40043E5389002301272A6E0F539E53890020F
:1014D400501272A6E0F53A9000B9E0F4042560F5E4
:1014E4003B9000F0E0FE9000B9E0F4042EF53CE5FA
:1014F40039B53A05853938800312123F85382C7581
:101504002B008041E5389002101272A6E0F539E50F
:10151400389002301272A6E0F53A9000C9E0F40463
:101524002560F53B9000B9E0FE9000C9E0F4042E7C
:10153400F53CE539B53A05853938800312123F8503
:10154400382C752B0022900101E0F53D7540117592
:101554005A02755B00AE52AF53E53D75F00FA4FD22
:10156400ACF0EDD39FEC9E4021E53D8E048F05FF4A
:10157400127265ED75F010A4FFAEF0E56075F01120
:1015840084FD7C00ED2FF53E800EE56075F011843E
:10159400FF7E00EF24F0F53E853E38E56075F011DE
:1015A40084AFF07E008F3B1211C585383FAE52AF39
:1015B40053900101E075F00FA4FDACF0EDD39FEC66
:1015C4009E4028755A02755B10853E381211C585F8
:1015D4003F3985383AAE52AF53E53D8E048F05FF4F
:1015E4001272908D3B853D3C12123FE5389008986D
:1015F400F8E4F0E8A3F0752C64752B002290010147
:10160400E0F53D754011755A02755B00AE52AF535B
:10161400E53D75F00FA4FDACF0EDD39FEC9E4021A9
:10162400E53D8E048F05FF127265ED75F010A4FF81
:10163400AEF0E56275F01184FD7C00ED2FF53E807F
:101644000EE56275F01184FF7E00EF24F0F53E850F
:101654003E38E56275F01184AFF07E008F3B1211C5
:10166400C585383FAE52AF53900101E075F00FA429
:10167400FDACF0EDD39FEC9E4028755A02755B10CB
:10168400853E381211C5853F3985383AAE52AF537D
:10169400E53D8E048F05FF1272908D3B853D3C1213
:1016A400123FE538900898F8E4F0E8A3F0E56C60A0
:1016B40017E56CC394FE50109000F5E0B402099055
:1016C40000E3E0D3940B5002801F900898E0FEA33F
:1016D400E0FFE56C12727574E78E048F05FF1272D9
:1016E40065900898ECF0A3EDF09000CBE0B4045FB3
:1016F400E56075F00484FF7E008F38E56075F004C2
:1017040084ADF07C008D3B754004755A01755B0017
:10171400E538C3943F50051211C580069001CFE00F
:10172400F538900898E0FEA3E0FFE538127275746E
:10173400328E048F05FF127265900898E0FEA3E0D4
:10174400FFEF2DFDEE3CFC900898ECF0A3EDF07556
:101754002C64752B0022900096E0B40146E5687570
:10176400F00A84FF7E008F38E56875F00A84ADF0D6
:101774007C008D3B75400A755A05755B00E538C3DE
:10178400941150051211C580069005A1E0F538AEFC
:101794002BAF2CE5382FFF50010E74641272B88EF3
:1017A4002B8F2C900097E0B40146E56975F00A840C
:1017B400FF7E008F38E56975F00A84ADF07C008DFA
:1017C4003B75400A755A05755B6CE538C394115036
:1017D400051211C5800690060DE0F538AE2BAF2C2E
:1017E400E5382FFF50010E74641272B88E2B8F2CC3
:1017F4009000A6E0B40249E56BC3944175F00584FA
:10180400FF7E008F38E56B75F00584ADF07C008DAC
:101814003B754005755A06755B00E538C394135053
:10182400051211C580069006A3E0F538AE2BAF2C47
:10183400E5382FFF50010E74641272B88E2B8F2C72
:101844009000E8E0B4020280030218F9E56075F044
:101854001584FF7E008F38E56075F01584ADF07C4B
:10186400008D3B754015755A03755BF4E538C394D8
:101874000B50051211C5800690048FE0F538E53849
:1018840075F0FFA4FFAEF09000E9E08E048F05FF31
:10189400127265ED90007FF0E56775F078A4FFAEF5
:1018A400F074FF8E048F05FF1272658C5A8D5B7481
:1018B400028C068D071200398F38AC5AAD5B740464
:1018C400FF1272908D3B754004755A06755B28E5CE
:1018D40038C3941D50051211C580069006D5E0F555
:1018E40038AE2BAF2CE5382FFF50010E7464127202
:1018F400B88E2B8F2C900095E0B4025DE56275F0F4
:1019040064A4FFAEF074081200398E5C8F5D740518
:101914008E048F05FF1272658D38AE5CAF5D740561
:101924008E048F05FF1272908D3B754005755A0524
:10193400755BDEE538C3941350051211C58006901B
:101944000681E0F538AE2BAF2CE5382FFF50010EA1
:1019540074641272B88E2B8F2C9000D7E0707F9035
:10196400005EE075F00A84FF7E008F3890005EE030
:1019740075F00A84ADF07C008D3B75400A755A05FC
:10198400755BC0E538C3940E50051211C5800690EE
:10199400065EE0F538E538900083F09000F6E0B498
:1019A400023C90005EE075F00A84FF7E008F389060
:1019B400005EE075F00A84ADF07C008D3B75400A52
:1019C400755A05755BCFE538C3940E50051211C5E1
:1019D400800690066DE0F538E538900084F022909A
:1019E400009EE0B401179008F3E0252CFFAE2B50C5
:1019F400010E9000F2E01272B88E2B8F2C9001161B
:101A0400E0B40114900117E0A852B80004955350B3
:101A140007E560C39561400280139000C0E0252C67
:101A2400FFAE2B50010E8E2B8F2C021E4A90009E6F
:101A3400E0B40306A22AB3B3400280509008FDE04C
:101A440070109008F6E0C39405A852B800069553A8
:101A5400400280109000C0E0252CFFAE2B50010EF8
:101A64008E2B8F2C9008FDE0600D9008F6E0A852B4
:101A7400B800069553400280109000C0E0252CFF6A
:101A8400AE2B50010E8E2B8F2C021E4A900098E034
:101A9400B402028003021E4A90009BE0602FE568B6
:101AA400D394464028900016E0FEA3E0FF9000D6B1
:101AB400E075F003A4FDACF0EFD39DEE9C400E90D6
:101AC40000FAE0A852B80005D395535003021E4A09
:101AD4009000CBE0B403028003021C9285625B7524
:101AE4005A009000A2E0A852B800049553500E90FA
:101AF40000A3E0A85AB80005D3955B5003021C8FDD
:101B0400E56275F002A4FFAEF074158E048F05FF34
:101B14001272658C068D07900620120048FEE0FFC5
:101B2400EE90009AE0FEEF8E0088F0A4FFAEF07411
:101B3400648E048F05FF1272658C5A8D5B90005E73
:101B4400E075F018A4FFAEF09000E1E08E048F057C
:101B5400FF1272658C068D07900638120048AE5A43
:101B6400AF5BE012727574648E048F05FF127265A8
:101B74008C5A8D5BE566A85AB80005D3955B500373
:101B8400021C06E566C3955BFFE4955AFE8E5A8FE8
:101B94005B7428BE00039F500C755B28755A007453
:101BA4000D90005FF0AE5AAF5B90009BE01272752F
:101BB40074288E048F05FF1272658C5A8D5B900811
:101BC40098E0FEA3E0FF740A8E048F05FF1272658D
:101BD4008D068C07AC5AAD5BCFCECF120003740ACE
:101BE4008E048F05FF1272658C5A8D5B900898E005
:101BF400FEA3E0FF1272C0900898EEF0A3EFF0028B
:101C04001C8FE566A85AB80004955B507EAE5AAFA7
:101C14005BE5661272B88E5A8F5B7428BE00039F10
:101C2400500C755B28755A00740D90005FF0AE5A25
:101C3400AF5B90009BE012727574288E048F05FFD1
:101C44001272658C5A8D5B900898E0FEA3E0FF74D5
:101C54000A8E048F05FF1272658D068C07AC5AAD8F
:101C64005BCFCECF120003740A8E048F05FF12726D
:101C7400658C5A8D5B900898E0FEA3E0FFEF2DFD84
:101C8400EE3CFC900898ECF0A3EDF0021E4A9000A4
:101C9400E3E08560F0A4FFAEF0740512727574077A
:101CA4001200398E5A8F5B9000A2E0A852B800044B
:101CB400955350129000A3E075F002A4FDACF0EF30
:101CC400C39DEE9C4003021E4AE56075F00B84FF41
:101CD4007E00900620120048FEE0FFEE90009AE09D
:101CE400FEEF8E0088F0A4FFAEF074648E048F05BE
:101CF400FF1272658C5A8D5B90005EE075F018A43B
:101D0400FFAEF09000E1E08E048F05FF1272658C47
:101D1400068D07900638120048AE5AAF5BE0127287
:101D24007574648E048F05FF1272658C5A8D5BE5A1
:101D340066A85AB80005D3955B5003021DC1E56639
:101D4400C3955BFFE4955AFE8E5A8F5B7428BE00E0
:101D5400039F500C755B28755A00740D90005FF05A
:101D6400AE5AAF5B90009BE012727574288E048F9C
:101D740005FF1272658C5A8D5B900898E0FEA3E013
:101D8400FF740A8E048F05FF1272658D068C07ACF2
:101D94005AAD5BCFCECF120003740A8E048F05FFB9
:101DA4001272658C5A8D5B900898E0FEA3E0FF12D6
:101DB40072C0900898EEF0A3EFF0021E4AE566A800
:101DC4005AB80004955B507EAE5AAF5BE56612725A
:101DD400B88E5A8F5B7428BE00039F500C755B2825
:101DE400755A00740D90005FF0AE5AAF5B90009B83
:101DF400E012727574288E048F05FF1272658C5A76
:101E04008D5B900898E0FEA3E0FF740A8E048F05B2
:101E1400FF1272658D068C07AC5AAD5BCFCECF1224
:101E24000003740A8E048F05FF1272658C5A8D5B51
:101E3400900898E0FEA3E0FFEF2DFDEE3CFC900837
:101E440098ECF0A3EDF0229000F6E0B4027BE5609C
:101E540075F00884FF7E008F38E56075F00884AD66
:101E6400F07C008D3B754008755A01755BE0E538E0
:101E7400C3943F50051211C5800690028FE0F538D7
:101E8400E53890089AF8E4F0E8A3F090089AE0FEA8
:101E9400A3E0FFAC2BAD2C12000374648E048F05F9
:101EA400FF12726590089AECF0A3EDF0900093E0B5
:101EB4008C068D0712727574648E048F05FF12727E
:101EC4006590089AECF0A3EDF0900898E0FEA3E08A
:101ED400FFAC2BAD2C12000374648E048F05FF122B
:101EE4007265900898ECF0A3EDF0900093E08C06F6
:101EF4008D0712727574648E048F05FF12726590DB
:101F04000898ECF0A3EDF0A204401DAE52AF537458
:101F140005BE00039F5002D204E562D394CC40086E
:101F2400D202741190005FF0229000F5E0B4020830
:101F34009000E3E0640B60028045900898E0FEA303
:101F4400E0FFE56C12727574E78E048F05FF127260
:101F540065900898ECF0A3EDF09000F6E0B4021F51
:101F640090089AE0FEA3E0FFE56C12727574E78EA8
:101F7400048F05FF12726590089AECF0A3EDF090BF
:101F840000B5E05402601B9000ACE0A852B8001207
:101F9400D39553400DA204B3B35007E562C3949A9A
:101FA4004002805FAE35AF369000AAE075F002A41F
:101FB400FDACF0EF2DFDEE3CFC74022DFD50010C48
:101FC400E562BC003ED39D403A754401A2314033E2
:101FD4009000ABE075F05EA4FDACF07405FF1272E6
:101FE400658C5C8D5D124A42900898E0FEA3E0FF88
:101FF4009000ABE02FFF50010E900898EEF0A3EF95
:10200400F0D231E562A835B8000495365002C231E9
:10201400856236753500E54470030221239001087A
:10202400E0C395445003022115900118E0C39402C3
:1020340040030220BFE56875F00A84FF7E00900526
:1020440090120048E0F55B755A00AE5AAF5B900001
:10205400ABE012727574648E048F05FF1272658C86
:102064005C8D5D900108E004C395448C068D0712D5
:102074007275900108E08E048F05FF1272658C5C06
:102084008D5D900898E0FEA3E0FFEF2DFDEE3CFC93
:10209400900898ECF0A3EDF09000F6E0B4021A90EA
:1020A400089AE0FEA3E0FFAA5CAB5DEF2BFBEE3ADF
:1020B400FA90089AEAF0A3EBF08056900108E00445
:1020C400C39544854CF0A4FFAEF0900108E08E0463
:1020D4008F05FF1272658C5C8D5D900898E0FEA3FD
:1020E400E0FFEF2DFDEE3CFC900898ECF0A3EDF042
:1020F4009000F6E0B4021A90089AE0FEA3E0FFAA6A
:102104005CAB5DEF2BFBEE3AFA90089AEAF0A3EB96
:10211400F00544900108E0C39544500375440090D1
:1021240000B5E05401601B9000A9E0A852B8001269
:10213400D39553400DA204B3B35007E560C394CCC8
:10214400400280609000A7E075F003A4FFAEF0E5C4
:10215400412FFF50010E74032FFF50010EE560BEA6
:102164000042D39F403E754501A23140379000A8FC
:10217400E075F05EA4FFAEF074058E048F05FF12C7
:1021840072658C5C8D5D124A42900898E0FEA3E073
:10219400FF9000A8E02FFF50010E900898EEF0A3E6
:1021A400EFF0D231E560C395415002C23185604100
:1021B400E54570030222BD900109E0C39545500333
:1021C4000222AF900118E0C394024003022259E5B1
:1021D4006875F00A84FF7E00900590120048E0F5CF
:1021E4005B755A00AE5AAF5B9000A8E0127275742A
:1021F400648E048F05FF1272658C5C8D5D900109FD
:10220400E004C395458C068D07127275900109E0B0
:102214008E048F05FF1272658C5C8D5D900898E0CA
:10222400FEA3E0FFEF2DFDEE3CFC900898ECF0A33C
:10223400EDF09000F6E0B4021A90089AE0FEA3E0F4
:10224400FFAA5CAB5DEF2BFBEE3AFA90089AEAF03A
:10225400A3EBF08056900109E004C39545854DF049
:10226400A4FFAEF0900109E08E048F05FF127265A1
:102274008C5C8D5D900898E0FEA3E0FFEF2DFDEEF1
:102284003CFC900898ECF0A3EDF09000F6E0B4026A
:102294001A90089AE0FEA3E0FFAA5CAB5DEF2BFB6B
:1022A400EE3AFA90089AEAF0A3EBF005459001099A
:1022B400E0C395455003754500900898E0FEA3E0FF
:1022C400FF9000BAE0BE00039F500D9000BAE0906A
:1022D4000898F8E4F0E8A3F09000F6E0B402129055
:1022E400089AE0FEA3E0FF9000BAE0BE00059F401C
:1022F40002800D9000BAE090089AF8E4F0E8A3F0A8
:10230400229000F6E0B401028003022453A204B335
:10231400500302243A9000C1E0B4017A900898E096
:10232400FEA3E0FFAC52AD53120003743C8E048F45
:1023340005FF1272659000D1E0BC00159D4012901B
:102344000898E0FEA3E0FF9000D3E0BE00039F5096
:1023540002D203900898E0FEA3E0FFAC52AD531202
:102364000003743C8E048F05FF1272659000D1E067
:10237400C3940ABC001AD39D4016900898E0FEA3AB
:10238400E0FF9000D3E0C39405BE0004D39F500245
:102394008002C203807A900898E0FEA3E0FFAC526A
:1023A400AD5312000374788E048F05FF127265908A
:1023B40000D1E0BC00159D4012900898E0FEA3E017
:1023C400FF9000D3E0BE00039F5004D203804190ED
:1023D4000898E0FEA3E0FFAC52AD531200037478FA
:1023E4008E048F05FF1272659000D1E0C3940ABC7D
:1023F400001AD39D4016900898E0FEA3E0FF9000D9
:10240400D3E0C39405BE0004D39F50028002C203EC
:10241400A203B34021900898E0FEA3E0FF9000D20D
:10242400E012727574648E048F05FF127265900851
:1024340098ECF0A3EDF0A203B3400CA2354006746F
:102444002490005FF0D235A2034002C2358002C25C
:102454000390005AE06006A204B3B34002801990CE
:102464000898E0FEA3E0FF90005AE02FFF50010E11
:10247400900898EEF0A3EFF0A201B34006A202B3D5
:10248400B3500990001EE4F0A3F0802D900898E06A
:10249400FEA3E0FF7400D39F74019E40119008983E
:1024A400E0F8A3E090001EC8F0A3C8F0800B74FF0E
:1024B40090001EF8E4F0E8A3F09000D8E0C3940480
:1024C400400C9008FAE0C3940240030225AD90004A
:1024D400C1E0B40147900898E0FEA3E0FF745E12E7
:1024E400727574058E048F05FF127265900898EC5E
:1024F400F0A3EDF09000F6E0B4021F90089AE0FE1D
:10250400A3E0FF745E12727574058E048F05FF12CA
:10251400726590089AECF0A3EDF08045900898E07D
:10252400FEA3E0FF745E127275740A8E048F05FFB9
:10253400127265900898ECF0A3EDF09000F6E0B408
:10254400021F90089AE0FEA3E0FF745E1272757495
:102554000A8E048F05FF12726590089AECF0A3EDC1
:10256400F0900898E0FEA3E0FF7402BE000CD39F35
:102574004008752A02752900800A900898E0F52918
:10258400A3E0F52A90089AE0FEA3E0FF7402BE00DF
:102594000CD39F4008752E02752D00800A90089A6E
:1025A400E0F52DA3E0F52E8046900898E0FEA3E028
:1025B400FF7401BE000CD39F4008752A01752900E1
:1025C400800A900898E0F529A3E0F52A90089AE09B
:1025D400FEA3E0FF7401BE000CD39F4008752E01DA
:1025E400752D00800A90089AE0F52DA3E0F52E9051
:1025F400001CE529F0A3E52AF0A238B34009C20182
:1026040090001EE4F0A3F02290005EE0900390128C
:1026140072A6E0F54275436490005EE0FE9000CC43
:10262400E0D39E4037E56075F00884FF7E008F3864
:10263400E56075F00884ADF07C008D3B754008754D
:102644005A03755B96E538C3941F50051211C58073
:1026540006900445E0F5388538438035E56075F02B
:102664000884FF7E008F38E56075F00884ADF07C47
:10267400008D3B754008755A03755BB6E538C39405
:102684001F50051211C58006900465E0F5388538A1
:102694004322900102E0F53D754011755A04755BC3
:1026A40000AE52AF53E53D75F00FA4FDACF0EDD391
:1026B4009FEC9E4021E53D8E048F05FF127265ED6F
:1026C40075F010A4FFAEF0E56075F01184FD7C0098
:1026D400ED2FF53E800EE56075F01184FF7E00EF6E
:1026E40024F0F53E853E38E56075F01184AFF07E48
:1026F400008F3B1211C585383FAE52AF5390010293
:10270400E075F00FA4FDACF0EDD39FEC9E4028756E
:102714005A04755B10853E381211C5853F398538DA
:102724003AAE52AF53E53D8E048F05FF1272908D81
:102734003B853D3C12123F8538427543642290012B
:1027440002E0F53D754011755A04755B00AE52AF59
:1027540053E53D75F00FA4FDACF0EDD39FEC9E4026
:1027640021E53D8E048F05FF127265ED75F010A40E
:10277400FFAEF0E56275F01184FD7C00ED2FF53EAF
:10278400800EE56275F01184FF7E00EF24F0F53EC3
:10279400853E38E56275F01184AFF07E008F3B1200
:1027A40011C585383FAE52AF53900102E075F00F6A
:1027B400A4FDACF0EDD39FEC9E4028755A04755BE4
:1027C40010853E381211C5853F3985383AAE52AF6F
:1027D40053E53D8E048F05FF1272908D3B853D3C81
:1027E40012123F8538427543649000FDE0B40479C9
:1027F40090005EE0FE9000CCE0D39E4037E560752B
:10280400F00884FF7E008F38E56075F00884ADF031
:102814007C008D3B754008755A03755B96E538C39B
:10282400941F50051211C58006900445E0F53885C3
:1028340038438035E56075F00884FF7E008F38E505
:102844006075F00884ADF07C008D3B754008755AC6
:1028540003755BB6E538C3941F50051211C5800695
:10286400900465E0F53885384322900096E0B40181
:102874003BE56875F00A84FF7E008F38E56875F0E3
:102884000A84ADF07C008D3B75400A755A05755B72
:1028940012E538C3941150051211C580069005B392
:1028A400E0F538E5432538C39464F543900097E098
:1028B400B4013BE56975F00A84FF7E008F38E56951
:1028C40075F00A84ADF07C008D3B75400A755A059D
:1028D400755B7EE538C3941150051211C5800690CE
:1028E400061FE0F538E5432538C39464F543E54213
:1028F4002543F53790009EE0B402109008F2E025DD
:1029040037FE9000F2E0F4042EF5379000F5E0D3A2
:1029140094014040E56CC394E7501D74E7C3956C83
:10292400FE9008F4E08E00F5F0E884FF7E008F3816
:10293400E5372538F537801CE56CC394E7FE90082D
:10294400F4E08E00F5F0E884FF7E008F38E537C3AD
:102954009538F537A2044006E5422464F537E53797
:10296400D394644009E537C39464F537800375371D
:10297400009000CEE0C3953750069000CEE0F537C6
:1029840022D201900081E0A852B800049553503E31
:10299400900081E0A852B800049553500375370F96
:1029A400900081E004A852B8000495535003753791
:1029B40007900081E02402A852B800049553500205
:1029C400C201900081E06006740990005FF0C2309B
:1029D4007E017F009000D4E01272759000E3E08ED7
:1029E400048F05FF127265E560BC000CD39D40089E
:1029F400D238740A90005FF0900096E0B401099018
:102A040000D5E0C39568400280159000E7E0A85225
:102A1400B8000495535002C201740B90005FF0900B
:102A24000096E0B40107E568C394644002801D90F9
:102A3400012DE0600D90012DE0A852B800069553D9
:102A440040028008C201740B90005FF0A2014003B1
:102A5400753700C237900116E0B40114900117E0F5
:102A6400A852B8000495535007E560C3956140022D
:102A7400802A9000BFE0D3941D400B9000BFE0C3B8
:102A8400941EF5378003753700A2344008741590FE
:102A9400005FF0D237D234D232022B7FC232C2343A
:102AA40090009EE0B40306A22AB3B34003022B7F36
:102AB4009008F6E0C39405A852B800049553500654
:102AC4009008FDE06002801F9000BFE0D3941D4099
:102AD4000B9000BFE0C3941EF53780037537007474
:102AE4000C90005FF0D2379008F6E0A852B80004CA
:102AF400955350069008FDE07002801F9000BFE0DF
:102B0400D3941D400B9000BFE0C3941EF53780039F
:102B1400753700740C90005FF0D2379008F6E0A887
:102B240052B80004955350319000DDE0B40228D22D
:102B3400309008FCE0FE9008FDE0D39E500690081B
:102B4400FDE0700280099008FCE4F0C23080069039
:102B540008FCE004F08002C2019008F6E02405A815
:102B640052B80004955350139000DDE0B4020A906B
:102B740008FDE07002D2308002C201A22FB34027C8
:102B84009000BFE0D3941D400B9000BFE0C3941E9F
:102B9400F5378003753700A2334006741090005F48
:102BA400F0D233D2378002C23385376D9000BFE054
:102BB400D3941D401890008DE02537FE90005EE010
:102BC40075F01E84FC7F00EE2CF5378037A237B3F6
:102BD400401690008DE0FE90005EE075F01E84FCCF
:102BE4007F00EE2CF537801C90008FE02537FE9097
:102BF400008DE02EFE90005EE075F01E84FC7F00E8
:102C0400EE2CF537A238B34005D230756D00229012
:102C1400005EE075F00584FF7E008F3890005EE072
:102C240075F00584ADF07C008D3B754005755A0345
:102C3400755BD69000E1E01475F00584FF7E00E535
:102C440038BE00039F50051211C5800BE53890046F
:102C5400661272A6E0F538E5389008F5F09008F5AC
:102C6400E0FE9000D0E0C39E50089000D0E09008B1
:102C7400F5F09000BFE0D3941D401E9008F5E0FEEF
:102C840090008DE02EFE90005EE075F01E84FC7FC7
:102C940000EE2C9008F5F0803FA237B34018900066
:102CA4008DE0FE90005EE075F01E84FC7F00EE2C4B
:102CB4009008F5F080229008F5E0FE90008FE02E59
:102CC400FE90008DE02EFE90005EE075F01E84FC08
:102CD4007F00EE2C9008F5F022900096E0B40136C7
:102CE400E56875F00A84FF7E00900590120048E0C4
:102CF400F547E547D394644010E547C3946475F001
:102D04000F84FF7E008F4780037547009000B3E077
:102D14002547F54780069000B3E0F54722E568753E
:102D2400F00A84FF7E00900590120048E0C3946985
:102D34004007E568D3946440559000FDE0C39403D4
:102D44005026900892E0FEA3E0FF7404120039E5D7
:102D540060127275740F8E048F05FF1272659008ED
:102D640090ECF0A3EDF08024900892E0FEA3E0FF45
:102D74007404120039E562127275740F8E048F05A3
:102D8400FF127265900890ECF0A3EDF0800F9008AC
:102D940092E0F8A3E0900890C8F0A3C8F0A2044021
:102DA4001A900892E0FEA3E0FF7403127275740196
:102DB400120039900890EEF0A3EFF09000A6E0B472
:102DC4000262E56BC3944175F00584FF7E008F3881
:102DD400E56B75F00584ADF07C008D3B75400575A1
:102DE4005A06755B14E538C3941750051211C58053
:102DF400069006B7E0F538900890E0FEA3E0FF7473
:102E04000A8E048F05FF127265E5388C068D071251
:102E14007275740A8E048F05FF127265900890EC27
:102E2400F0A3EDF0900890E0FEA3E0FF900896E098
:102E3400FCA3E0FDEDD39FEC9E400F900896E0F8D4
:102E4400A3E0900890C8F0A3C8F022E50875F00448
:102E5400A4FFAEF09006D3120048E0903CE8F828B6
:102E64002873804C85537480479000E3E08560F0BC
:102E7400A4FFAEF074081200398F74803385627435
:102E8400802E85687480298569748024856A74809D
:102E94001F856B74801A856C748015856774801027
:102EA400856674800B856D74800690001FE0F57450
:103CE800022E66022E68022E6D022E81022E860298
:103CF8002E8B022E90022E95022E9A022E9F022EB5
:073D0800A4022EA9022EAE59
:102EB400E50875F004A4FFAEF09006D4120048E5CE
:102EC4000875F004A4FFAEF0E0FC9006D5120048AB
:102ED400ECFEE0FFEEC39F4003022FBCE50875F053
:102EE40004A4FFAEF09006D3120048E0B40441E518
:102EF4000875F004A4FFAEF09006D5120048E0C3B4
:102F04009574500AE508F50CD39239123EB1E508E0
:102F140075F004A4FFAEF09006D4120048E0D395F7
:102F240074400AE508F50CC39239123EB1022FBA77
:102F3400E50875F004A4FFAEF09006D4120048E052
:102F4400C395745015E50875F004A4FFAEF090061F
:102F5400D5120048E0D395745002800AE508F50CB8
:102F6400D39239123EB1E50875F004A4FFAEF09097
:102F740006D4120048E0D395745015E50875F004A2
:102F8400A4FFAEF09006D5120048E0C39574500A31
:102F9400E508F50CC39239123EB19006DBE0B401AA
:102FA400099000EFE0D395625002800A7402F50C98
:102FB400C39239123EB1806AE50875F004A4FFAEED
:102FC400F09006D4120048E0D395744015E50875D6
:102FD400F004A4FFAEF09006D5120048E0C3957447
:102FE4004002800AE508F50CC39239123EB1E508A7
:102FF40075F004A4FFAEF09006D4120048E0C39527
:10300400744015E50875F004A4FFAEF09006D512DF
:103014000048E0D39574400AE508F50CD3923912C0
:103024003EB122AE2FAF3074C9BE000CD39F40080E
:10303400782F1272C8023141753001752F00AE52DB
:10304400AF53E547BE000DD39F40099000C5E0D3C0
:10305400954840028023754800E547C39553F574AD
:103064009000C8E0D395464008E5462574F54680AF
:10307400069000C8E0F546800205489000A1E0D320
:103084009562401CE560C395614015AE52AF53E5AF
:1030940047BE00039F50099000C6E0D39549400203
:1030A400806E9008F7E0A852B80004955350037559
:1030B4004B009008F7E0A852B8000BD39553400694
:1030C400E5539008F7F0E54B7041E553C39547F598
:1030D40074E574D3940540037574059000C7E0C388
:1030E40095465007E574C3954640028009E546C3FA
:1030F4009574F54680069000C7E0F5469000C7E059
:10310400D3954640069000C7E0F546754900800215
:103114000549E54B70169000A1E0C39562500DE59A
:10312400472405A852B8000695534002800F90002A
:10313400B4E0F546754B0174789008F7F022AE2F91
:10314400AF3074E9D39F74039E4008782F1272C87D
:103154000232FB753001752F00754632A22B403DBB
:10316400E54875F00284AFF07E00EF4E70057546B9
:103174001980037546329000B4E075F002A4FFAEE6
:10318400F0E548BE0006D39F4002D22B0548754B9C
:103194000374789008F7F0754A000232E2AE52AF39
:1031A40053E5476F4E70030232E2E547BE000DD38C
:1031B4009F40099000C5E0D395484002800F7548B0
:1031C40000E54BC394035003754619800DE547C3CE
:1031D4009553F574E5482574F5489000A1E0D3951E
:1031E40062400E9008F7E0A852B80007D395534008
:1031F40002800C054A9000B4E0B54A03754B00E523
:103204004BB40306A204B3B34002800A054AE54A5C
:10321400B43C03754B02E54BB402299008F7E0A8CF
:1032240052B8000ED395534009E5539008F7F07552
:103234004A009000A1E0C395625009754A00747871
:103244009008F7F0E54B705A9000A1E0D3956240E6
:103254001CE560C395614015AE52AF53E547BE000F
:10326400039F50099000C6E0D39549400280087539
:10327400490075464B8028E553C39547F574E574BA
:10328400D3940540037574059000A1E0D395624082
:1032940008E5492574F5498006E5492406F549758C
:1032A4004A00E54B70169000A1E0C39562500DE50D
:1032B400472405A852B80006955340028003754B75
:1032C40001E54BB40118754619054A9000B4E0B500
:1032D4004A06754B02754A0074789008F7F0A2020A
:1032E400B34003754632E54675F00AA4FFAEF0908C
:1032F400089CEEF0A3EFF022E570903D0FF828282B
:1033040073023CA8900099E0700302362C9000CF21
:10331400E0B4010280030234BF90005CE0655F60AA
:1033240009E553455260030234BC7E017F00E5BECB
:10333400127275E5BD2FFF50010E8E5A8F5B9001FE
:1033440034E075F010A4FDACF08C5C8D5DEFD39D82
:10335400EE9C40091272C08E5A8F5B8006755B002A
:10336400755A00AE5AAF5B740E1272759000C4E0C9
:103374008E048F05FF1272659008A0ECF0A3EDF0A7
:10338400E56C600FE56CC394FE50089000F5E064B2
:1033940002600280649000E3E0B40B1F9008A0E098
:1033A400FEA3E0FF74E7127275E56C8E048F05FFCF
:1033B4001272659008A0ECF0A3EDF09000E3E0D366
:1033C400940B40089000CBE064046002802B9008CA
:1033D400A0E0FEA3E0FF9008A4E0FCA3E0FDEFD38F
:1033E4009DEE9C400D1272C09008A0EEF0A3EFF089
:1033F40080079008A0E4F0A3F09008A0E0FEA3E00A
:10340400FFEFD39400EE94014008D2387426900064
:103414005FF0A238B3B3502C7E057F009000E3E048
:103424008E048F05FF1272659008A0E0FEA3E0FFF2
:10343400EFC39DEE9C400FAC52AD53740FBC00041F
:10344400D39D50028002C238900099E0B4022790C4
:1034540008A2E0FEA3E0FF9008A0E0FCA3E0FDEFDB
:103464002DFDEE3CFC74018C068D0712003990088A
:10347400A0EEF0A3EFF09008A0E0FEA3E0FF900818
:10348400A2E0FCA3E0FDEDD39FEC9E4004D22E808D
:1034940002B22E9008A0E0F8A3E09008A2C8F0A31E
:1034A400C8F09000CBE064016006A22EB3B34002E2
:1034B40080069008A1E0F56002362AD22E7E017FB4
:1034C40000E5BE127275E5BD2FFF50010E8E5A8FB6
:1034D4005B900134E075F010A4FDACF08C5C8D5D64
:1034E400EFD39DEE9C40091272C08E5A8F5B80060A
:1034F400755B00755A00AE5AAF5B740E127275900C
:1035040000C4E08E048F05FF1272659008A0ECF0F1
:10351400A3EDF0E56C600FE56CC394FE50089000D9
:10352400F5E06402600280649000E3E0B40B1F9055
:1035340008A0E0FEA3E0FF74E7127275E56C8E0448
:103544008F05FF1272659008A0ECF0A3EDF09000D7
:10355400E3E0D3940B40089000CBE0640460028065
:103564002B9008A0E0FEA3E0FF9008A4E0FCA3E0F9
:10357400FDEFD39DEE9C400D1272C09008A0EEF0BA
:10358400A3EFF080079008A0E4F0A3F09008A0E077
:10359400FEA3E0FFEFD39400EE94014008D2387408
:1035A4002690005FF0A238B3B3502C7E057F0090C4
:1035B40000E3E08E048F05FF1272659008A0E0FE20
:1035C400A3E0FFEFC39DEE9C400FAC52AD53740FCC
:1035D400BC0004D39D50028002C238900099E0B42C
:1035E40002279008A2E0FEA3E0FF9008A0E0FCA35D
:1035F400E0FDEF2DFDEE3CFC74018C068D071200FE
:10360400399008A0EEF0A3EFF09008A0E0F8A3E052
:103614009008A2C8F0A3C8F09000CBE06401600653
:103624009008A1E0F5608003756000900095E0705B
:10363400067570030232FC75BB18023CA8023CA854
:10364400900095E070030237B57E017F00E5BE125D
:103654007275E5BD2FFF50010E8E5A8F5B9000DB13
:10366400E0B4010F7E0F7FFFAC5AAD5B1272C08EC7
:103674005A8F5B900100E0B40245AE5AAF5B9000F4
:1036840028E0FCA3E0FDEDD39FEC9E400A900028C7
:10369400E55AF0A3E55BF0AE5AAF5B90002AE0FC7C
:1036A400A3E0FDEFD39DEE9C400A90002AE55AF07A
:1036B400A3E55BF0AE5AAF5B74041200398F6290DD
:1036C4000100E0704CAE5AAF5B900028E0FCA3E030
:1036D400FDEFD39DEE9C40091272C08E5A8F5B8021
:1036E40006755B00755A00AE5AAF5B7410127275A2
:1036F4009000FFE08E048F05FF1272658C5A8D5B7B
:1037040074FFBC0009D39D4005855B62800375622C
:10371400FE9000CBE0B4010280030237B3A204B3ED
:10372400B3500E90009FE0A852B80005D3955350B3
:103734000280719000DCE08562F0A4FFAEF0746456
:103744008E048F05FF1272658C5A8D5BE56C6016D2
:10375400E56CC394FE500F9000F5E0B402089000AD
:10376400E3E0640B60028017AE5AAF5B74E7127239
:1037740075E56C8E048F05FF1272658C5A8D5BAEF5
:103784005AAF5B9008A0E0FCA3E0FDEDD39FEC9E54
:103794004005855B60800BA22EB340069008A1E033
:1037A400F560800BA22EB340069008A1E0F560807E
:1037B40003756200900098E070067570050232FC93
:1037C40075BB19023CA8023CA8900098E070030263
:1037D400389CE55FD3955E400302389A900026E05A
:1037E400FEA3E0FFE5661272B8900026EEF0A3EFA8
:1037F400F0900105E0B402247E017F00E5BE127260
:1038040075E5BD2FFF50010E8F048E057E0F7FFFDF
:10381400CDCCCD1272C08E5A8F5B80147E017F0096
:10382400E5BE127275E5BD2FFF50010E8E5A8F5BF7
:10383400900105E07017AE5AAF5B740A127275748A
:10384400518E048F05FF1272658D668019AE5AAFD2
:103854005B740A1272758F048E057E017F95CDCC40
:10386400CD1271638F66E566D39464400375666414
:10387400900026E0FEA3E0FFE5662FFF50010E90C6
:103884000026EEF0A3EFF090009CE0048E048F0578
:10389400FF1272658D6680037566329000E8E070F1
:1038A400067570070232FC75BB13023CA8023CA8E3
:1038B4009000E8E0604A7E017F00E5BE127275E583
:1038C400BD2FFF50010E8E5A8F5B74041200398F86
:1038D400679000EAE08567F0A4FDACF07464FF1221
:1038E40072658D679000E9E08567F0A4FFAEF0741F
:1038F400FF8E048F05FF127265ED900080F0800347
:10390400756700900096E070067570090232FC75C8
:10391400BB17023CA8023CA8900096E0B4010280C8
:10392400030239B07E017F00E5BE127275E5BD2F3A
:10393400FF50010E8E5A8F5B9008F8E060199008D2
:10394400F8E014906C8212008CE493FC740193FDF3
:10395400EDC39FEC9E400280069008F8E014F090BE
:1039640008F8E0C394B3501DAE5AAF5B9008F8E07A
:1039740004906C8212008CE493FC740193FDEFC3F9
:103984009DEE9C400280069008F8E004F09008F850
:10399400E0FE9000BCE08E0088F0A4FFAEF07464FA
:1039A4008E048F05FF1272658D6880037568009020
:1039B4000097E0700675700B0232FC75BB16023C72
:1039C400A8023CA8900097E0B401028003023A5C8C
:1039D4007E017F00E5BE127275E5BD2FFF50010E1A
:1039E4008E5A8F5B9008F9E060199008F9E0149002
:1039F4006DEC12008CE493FC740193FDEDC39FEC19
:103A04009E400280069008F9E014F09008F9E0C3A3
:103A140094B3501DAE5AAF5B9008F9E004906DEC7E
:103A240012008CE493FC740193FDEFC39DEE9C4063
:103A34000280069008F9E004F09008F9E0FE900096
:103A4400C2E08E0088F0A4FFAEF074648E048F058B
:103A5400FF1272658D69800375690075BB1F023C96
:103A6400A8023CA87E017F00E5BE127275E5BD2F59
:103A7400FF50010E8E5A8F5B740912727574E68EB4
:103A8400048F05FF1272658D6B90009EE0700675C1
:103A9400700F0232FC75BB15023CA8023CA89000D2
:103AA4009EE07003023BF37E017F00E5BE12727557
:103AB400E5BD2FFF50010E8E5A8F5B74041200393E
:103AC4008F6A90009EE0B401159000F2E0856AF0E0
:103AD400A4FFAEF07407120039EF9008F3F09000E1
:103AE4009EE0B402159000F2E0856AF0A4FFAEF007
:103AF4007407120039EF9008F2F090009EE0B403CE
:103B0400028003023BD69000DFE07052E56AC39462
:103B140019500FD22A9000BEE09008F6F09008FBEE
:103B2400E4F0E56AD394644004A22A4002802D9014
:103B340008FBE004F09008FBE0FE900131E0B506DC
:103B44000B9008F6E004F09008FBE4F09008F6E02F
:103B540064966006900131E07002C22A806390008E
:103B6400BEE070349000F2E0856AF0A4FFAEF07419
:103B7400FF8E048F05FF127265ED9008F6F0AE52C9
:103B8400AF53741EBE0006D39F4002D22AE562D30F
:103B940094E54002C22A8029E56AC3940A500DAE16
:103BA40052AF53741EBE0004D39F50028002D22A27
:103BB400E562D394E54002C22A9000BEE09008F684
:103BC400F09008F6E0C39405500674059008F6F0EA
:103BD400C22F90009EE0B40414E56AC39419500205
:103BE400D22FE56AD394324002C22FC22A800375D1
:103BF4006A009000F5E070067570110232FC75BB26
:103C040014023CA8023CA89000F5E07003023C9525
:103C14007E017F00E5BE127275E5BD2FFF50010ED7
:103C24008E5A8F5B900135E075F010A4FDACF08CDA
:103C34005C8D5DEFD39DEE9C40091272C08E5A8F4D
:103C44005B8006755B00755A00AE5AAF5B740E124A
:103C540072759000FCE08E048F05FF1272658C5C17
:103C64008D5D74FFBC00039D5005756CFF8003855A
:103C74005D6CE56C75F00BA4FFAEF09000E3E08E94
:103C8400048F05FF1272659008A4ECF0A3EDF08098
:103C940003756C00900099E0600575BB1A8003758C
:043CA400BB188000C9
:103D0F000233050233080236410236440237CA0233
:103D1F0037CD0238B10238B402391902391C0239D1
:103D2F00C50239C8023A65023A68023A9F023AA2BE
:093D3F00023C08023C0B023CA806
:103CA800E57075F00284AFF07E00EF4E7002D2EC42
:033CB80005702272
:0972A6002582F5825002058322C5
:0F008C0025E050020583258250020583F582226C
:10724400EF2F500205832582F582E5833E2EF583D8
:017254002217
:1072B800CFC39FFF50011E22C3EF9DFFEE9CFE220D
:0872C8000806B60002180622B8
:0D728300A3E004F0700612729CE004F022FB
:0E003900048007C3CE13CECF13CFD5E0F6223E
:10716300BC000FBE0008ED8FF084FFADF022E4FEFB
:10717300FF22BE000DEF60FE54F0606F20E70302B4
:107183007219EAC0E0EBC0E078017A0075F001EE15
:1071930020E710EF25E0FFEE33FE0AC5F023C5F02C
:1071A30030E7F0EA5407F9096A7A007B00600108C6
:1071B300C3EC9E40167004ED9F4010ED9FFDEC9EC6
:1071C300FCE5F0CA4ACA03F5F08005E5F003F5F0E3
:1071D300C3EE13FEEF13FFD9D77908CACBCAD8D0B1
:1071E300EAFEEBFFD0E0FBD0E0FA22EC8FF084FC68
:1071F300ED54F045F0C48FF084FEEDC454F045F037
:10720300C48FF084FDEEC4FE54F02DFFEE540F3C0A
:10721300FEADF07C0022790078008FF0EC7E082030
:10722300E70DC3CD33CD33C933C9C833C8DEF084CA
:1072330049F9E5F08FF0BE00E6FD7C00E9FFE8FECA
:017243002228
:0E727500F88FF0A4FFE5F0CE88F0A42EFE22E4
:10000300EF8DF0A4F9A8F0EF8CF0A428F8EE8DF0B2
:06001300A428FEE9FF2213
:10725500600D782B02725F007830D8FED5E0F822F9
:10726500EEC0E07E00127163EFFDEEFCD0E0FE2281
:0C729000EEC0E07E00127163D0E0FE2230
:03001B0002001EC2
:0300530002005652
:03009B00020071EF
:030000000272AFDA
:0972AF0075817675D000024BAC2C
:0B004800E5822FF582E5833EF5832260
:0A729C000582D582021583158222B7
:10001E00C0E0C0F0C083C082C0D075D000124B2E9D
:0B002E00D0D0D082D083D0F0D0E032E0
:10005600C0E0C0F0C083C082C0D075D000124B3162
:10006600D0D0D082D083D0F0D0E032C0E0C0F0C093
:1000760083C082C0D075D000124B6ED0D0D082D053
:0600860083D0F0D0E0324F
:00000001FF
